:100000000C942C050C9424290C9449050C94490556
:100010000C9449050C9449050C9449050C94490528
:100020000C9449050C9449050C9413310C94E5315A
:100030000C945E2B0C9449050C9449050C944905CD
:100040000C9449050C9449050C9449050C944905F8
:100050000C9449050C94022C0C9449050C94490508
:100060000C9449050C9449050C9449050C944905D8
:100070000C9449050C9449050C9449050C944905C8
:100080000C9449050C9449050C9449050C944905B8
:100090000C9449050C9449050C9449050C944905A8
:1000A0000C9449050C9449050C944905B909B90902
:1000B000E509E5094D0A780B780B780B6B0A040B00
:1000C000150B150B52327932713379327133C532D7
:1000D000E83271333F334E3329001E001F002000E9
:1000E000210022002B0014001A0008001500170040
:1000F000E00004001600070009000A00E1001D00EE
:100100001B00060019000500000000004A00E30083
:10011000A85D28002A0027002600250024002300CF
:100120004C00130012000C0018001C0034003300B7
:100130000F000E000D000B00E50038003700360000
:1001400010001100000000004D00E600A95D2C0029
:1001500035021E021F02200221022202005C1E0044
:100160001F002000210022004C00010050004F0021
:1001700052002F00C15C01000100010051002F025C
:10018000000000002602010001004C002A002702A6
:100190002602250224022302010027002600250052
:1001A0002400230031022E025E005D005C0030005E
:1001B00001002D005B005A005900300200000000D1
:1001C0002702620001004C0045003A003B003C0061
:1001D0003D003E00C35C1E021F02200221022202DB
:1001E000C45CAC00AB00A9004B002D02A800AD0020
:1001F000AE00AA004E002D00000000002602010003
:1002000001000100440043004200410040003F0063
:100210000100270226022502240223023100CA5CC3
:10022000C85CC65C4A002E000100CB5CC95CC75CA0
:100230004D002E020000000001000100010001003D
:1002400001000100010001000100010001000100A6
:100250000100010001000100010001000100010096
:100260000100010001000100010001000100010086
:100270000000000001000100010001000100010078
:100280000100010001000100010001000100010066
:100290000100010001000100010001000100010056
:1002A0000100010001000100010001000000000048
:1002B000010001000100010044454255473A206415
:1002C000697361626C65642E0A0044454255473A81
:1002D00020656E61626C65642E0A000A002530326A
:1002E00058006C65645F7461736B3A20004F6E65F3
:1002F00073686F743A206163746976653A20256487
:100300000A000A0025303862003A200025303258B1
:10031000000A722F632030313233343536370A0009
:1003200054617267657420636F6E6E656374656493
:100330000D0A0054617267657420646973636F6E9F
:100340006E65637465642C207468726F74746C6974
:100350006E6720636F6E6E656374696F6E20617483
:1003600074656D7074730D0A004661696C65642074
:10037000746F20657865637574652025730A007253
:1003800067626C696768742074696D65722064695E
:100390007361626C652E0A007267626C69676874CB
:1003A0002074696D657220656E61626C65642E0AE9
:1003B000007267626C696768742073657420687383
:1003C00076205B4E4F454550524F4D5D3A20257586
:1003D0002C25752C25750A007267626C6967687434
:1003E0002073657420687376205B454550524F4DED
:1003F0005D3A2025752C25752C25750A00726762DB
:100400006C69676874207261696E626F77207365CA
:1004100074206873763A2025642C25642C25642C7E
:1004200025750A007267626C696768742064697375
:1004300061626C65205B454550524F4D5D3A2072BC
:1004400067626C696768745F636F6E6669672E6563
:100450006E61626C65203D2025750A007267626CD2
:100460006967687420656E61626C65205B45455004
:10047000524F4D5D3A207267626C696768745F63C2
:100480006F6E6669672E656E61626C65203D202522
:10049000750A007267626C6967687420746F6767B9
:1004A0006C65205B454550524F4D5D3A2072676246
:1004B0006C696768745F636F6E6669672E656E61ED
:1004C000626C65203D2025750A007267626C696761
:1004D0006874206D6F6465205B4E4F454550524FE8
:1004E0004D5D3A2025750A007267626C6967687411
:1004F000206D6F6465205B454550524F4D5D3A203D
:1005000025750A007267626C696768745F696E6955
:1005100074207267626C696768745F636F6E666986
:10052000672E6D6F6465203D20302E2057726974F0
:10053000652064656661756C742076616C756573A1
:1005400020746F20454550524F4D2E0A007267624D
:100550006C696768745F696E6974206565636F6E46
:10056000666967206973206E6F7420656E61626CC6
:1005700065642E0A007267626C696768745F696EF1
:100580006974207374617274210A007267626C6905
:100590006768745F696E69742063616C6C65642E52
:1005A0000A007267626C696768745F636F6E666980
:1005B000672E7370656564203D2025640A007267AC
:1005C000626C696768745F636F6E6669672E7661D7
:1005D0006C203D2025640A007267626C696768744C
:1005E0005F636F6E6669672E736174203D202564BA
:1005F0000A007267626C696768745F636F6E666930
:10060000672E687565203D2025640A007267686C56
:10061000696768745F636F6E6669672E6D6F646586
:10062000203D2025640A007267626C696768745F08
:10063000636F6E6669672E656E61626C65203D2032
:1006400025640A007267626C696768745F636F6E25
:1006500066696720454550524F4D3A0A0000047FB5
:100660003F1F643214643214783C1E1E140A0522A3
:1006700023252628292A2C2D2F3032333536383A97
:100680003B3D3E4042434547494A4C4E50515355ED
:1006900057595A5C5E6062646668696B6D6F71730E
:1006A0007577797B7D7F81838587898A8C8E90920F
:1006B0009496989A9C9E9FA1A3A5A7A8AAACAEAF1A
:1006C000B1B3B4B6B8B9BBBCBEBFC1C2C3C5C6C75F
:1006D000C9CACBCCCDCED0D1D2D2D3D4D5D6D7D710
:1006E000D8D9D9DADADBDBDBDCDCDCDCDCDDDDDD58
:1006F000DDDCDCDCDCDCDBDBDBDADAD9D9D8D7D754
:10070000D6D5D4D3D2D2D1D0CECDCCCBCAC9C7C600
:10071000C5C3C2C1BFBEBCBBB9B8B6B4B3B1AFAE3E
:10072000ACAAA8A7A5A3A19F9E9C9A9896949290E4
:100730008E8C8A89878583817F7D7B7977757371BC
:100740006F6D6B6968666462605E5C5A5957555399
:1007500051504E4C4A4947454342403E3D3B3A3852
:1007600036353332302F2D2C2A292826252322FFF7
:10077000AA7F55406261636B6C696768742073740B
:1007800065703A2025750A006261636B6C69676861
:10079000742064697361626C650A006261636B6CEA
:1007A0006967687420656E61626C650A00626163E6
:1007B0006B6C6967687420746F67676C653A202595
:1007C000750A006261636B6C6967687420646563B5
:1007D00072656173653A2025750A006261636B6C0E
:1007E0006967687420696E6372656173653A202574
:1007F000750A00000101010101010101010202026B
:1008000002020202020203030303030303030404BC
:100810000404040404050505050506060606060786
:100820000707070708080808090909090A0A0A0B3F
:100830000B0B0C0C0C0D0D0D0E0E0E0F0F0F1010E0
:100840001111111212131314141515161617171867
:100850001819191A1A1B1B1C1D1D1E1E1F202021D2
:100860002222232424252626272829292A2B2C2D19
:100870002D2E2F30313232333435363738393A3B3A
:100880003C3D3E3F404142434445464748494A4C2F
:100890004D4E4F50515354555658595A5B5D5E5FFB
:1008A000616264656668696B6C6D6F707273757791
:1008B000787A7B7D7E8082838587888A8C8E8F91F3
:1008C000939596989A9C9EA0A2A3A5A7A9ABADAF1D
:1008D000B1B3B5B7BABCBEC0C2C4C6C9CBCDCFD107
:1008E000D4D6D8DBDDDFE2E4E7E9EBEEF0F3F5F8B0
:1008F000FAFDFF0A002530325820006B6579626FDF
:100900006172645F7265706F72743A20005B735D30
:10091000005B575D005B535D005B525D005B445DB7
:10092000005B435D001C03490072006900730020F6
:10093000004B006500790062006F00610072006486
:100940000000000E034B0065006500620069006F47
:100950000000000403090409025B00030100A0FA7F
:100960000904000001030101000921110100012215
:10097000400007058103080001090401000103008C
:100980000000092111010001223200070582032025
:100990000001090402000203000000092111010006
:1009A000012222000705830320000107050303201D
:1009B0000001120100020000000810CB56120001D5
:1009C000010200010631FF0974A101097515002615
:1009D000FF009520750881020976150026FF009515
:1009E0002075089102C005010980A1018503190144
:1009F0002AB700150126B700950175108100C005C2
:100A00000C0901A101850419012AA002150126A0E3
:100A100002950175108100C005010906A1010507B5
:100A200019E029E715002501950875018102950156
:100A3000750881010507190029FF150026FF00959B
:100A400006750881000508190129059505750191AC
:100A500002950175039101C011241FBECFEFDAE0AA
:100A6000DEBFCDBF12E0A0E0B1E0ECE9F9E602C0E4
:100A700005900D92AA30B107D9F723E0AAE0B2E0C1
:100A800001C01D92A534B207E1F70E941E1B0C9411
:100A9000CC340C940000FF93EF93E0910A02F091A4
:100AA0000B02309709F00995EF91FF910895FC0131
:100AB0008591803011F0EFDFFBCF0895FF27E0E252
:100AC00030E247FF0CC0419597FF09C0EDE2609509
:100AD000709580959095611D711D811D911D27FF59
:100AE00002C0219530E350E2AA27660F771F881FC6
:100AF000991FAA1FA41710F0A41B63955A95A9F774
:100B0000AA3008F0A95FA05DAF93F3956115710558
:100B10008105910541F7ED3211F4EF93F395F2174A
:100B200018F43F93F395FBCF8F91B5DFFA95E1F77A
:100B30000895E991F9918591803021F0853219F07D
:100B4000AADFF9CF089520E0E89455915532C1F31A
:100B5000503311F4689455915A3348F4505390F33C
:100B6000220F022E220F220F200D250FF4CF0EF49C
:100B7000219589919991533619F3533729F15335BA
:100B800059F1BC0188279927E8945C3621F48991B2
:100B9000999168945591543639F446EF7EF077FF79
:100BA0000DC08FEF9FEF0AC055374AE039F0583536
:100BB00040E121F0523642E009F00895FF93EF93AF
:100BC0007DDFEF91FF91B7CFFF93EF93FC01819110
:100BD0008030B9F360DFFBCFFF93EF9368DFF1CF95
:100BE000DF93CF93CDB7DEB72596A3DFCF91DF910B
:100BF0000895CF93FB01883A2DE59207A1F020F4E8
:100C0000873A9D4549F031C0893A2DE5920771F048
:100C10008A3A9D45F9F029C0C281CC2339F180E0A0
:100C20000E9489061DC0C28181E002C0C28182E0AB
:100C3000CC2341F00E94BC0C43E062E081E00E94C2
:100C4000F7060EC00E94DD0C43E062E081E00E94E6
:100C5000F7060CC0C28183E0CC2321F00E94BC0CBB
:100C6000C0E004C00E94DD0C01C0C1E08C2FCF9118
:100C7000089581E008950C94F90508950C943D06BB
:100C80001F93CF93DF9300D000D01F92CDB7DEB774
:100C900049835A836B8330910D0289819A81311186
:100CA00014C0662359F0222349F00E94B30D182F77
:100CB000682F89819A810E945A0D03C00E94860D77
:100CC000182F69817A81812F04C00E94B30D698138
:100CD0007A810F900F900F900F900F90DF91CF912E
:100CE0001F910C94F114FC01262F408151816281E7
:100CF000738184810C94400681E00895CF93DF9343
:100D0000EC0160E00E947306BE01DF91CF910C946C
:100D10003E06CF92DF92EF92FF92C12CD12C76014A
:100D2000C39404C0CC0CDD1CEE1CFF1C8A95D2F7CA
:100D30008C2D0E946312C701B601FF90EF90DF90E7
:100D4000CF900C945C0C8F929F92AF92BF92CF92F7
:100D5000DF92EF92FF920F931F936B017C0181E072
:100D600090E0A0E0B0E04C015D0104C0880C991C4B
:100D7000AA1CBB1C4A95D2F7AC01BD0104C0440FAC
:100D8000551F661F771F2A95D2F7482959296A29C6
:100D90007B2904C0880F991FAA1FBB1F0A95D2F791
:100DA0008A019B010C211D212E213F214017510753
:100DB0006207730739F4BC01CD016C297D298E29A6
:100DC0009F290AC080959095A095B095BC01CD0152
:100DD0006C217D218E219F211F910F91FF90EF901B
:100DE000DF90CF90BF90AF909F908F9008950F931A
:100DF000382F262F60913602709137028091380289
:100E000090913902042F432F0E94A3060F910C9456
:100E1000960C0C94AA160C94A61608950E94040C25
:100E20000E940D072FEF84E39CE02150804090400A
:100E3000E1F700C000000C94282C0F931F93CF9370
:100E4000DF938C0161E00E947306EC01B8010E94FF
:100E50003B06882369F1B801CE010E94072588234B
:100E600039F1B801CE010E943128882309F1B80177
:100E7000CE010E9445268823D9F0B801CE010E94F8
:100E80008D278823A9F0B801CE010E94D52288239E
:100E900079F0F80182818823E1F1CF3D8CE5D80714
:100EA00081F160F4C115FCE5DF0721F40E940E0713
:100EB000C0E036C0C130DC4579F02BC0CC35EDE563
:100EC000DE0729F1CD35FDE5DF07F1F0CB35DD4556
:100ED00001F50E944A121DC080919C02C82FC09546
:100EE000C170C0FB80F980939C02CC2329F08AEC6E
:100EF00092E00E945705DCCF88EB92E00E945705F4
:100F00000FC00E94FD12D4CF0E94411202C00E9465
:100F10004D12C801DF91CF911F910F910C943906AA
:100F20008C2FDF91CF911F910F9108950E94412B3B
:100F300080E00E943C250C94C6070E94BF230E94BB
:100F4000C9070C94472B8295982F937344E0949F84
:100F5000900111248C7C86958695282B822F85758F
:100F6000880F2A7A2695822B089508950C94B50748
:100F700081E008950C94B8070895CF93C82F0E947C
:100F8000B6078C2F0E94BA07CF91089580E00C9489
:100F9000BD070E944F2A0C94BD07CF930E944F2A91
:100FA000C82F80910C02C81741F1C0930C028091A8
:100FB0009C0282FF1EC080FF04C082EE92E00E946D
:100FC000570580919C0280FF0CC01F92CF938DED3E
:100FD00092E09F938F930E94F0050F900F900F90D7
:100FE0000F9080919C0280FF04C08BED92E00E94E4
:100FF00057058C2FCF910C94BD07CF910895CF93B7
:10100000DF93CDB7DEB72B970FB6F894DEBF0FBED8
:10101000CDBF4F83588769877A878B8761110E947C
:1010200079119E012F5F3F4F86E0F90111928A9559
:10103000E9F785E0FE013796D90101900D928A9576
:10104000E1F789819A814C815D81452B31F09F3F89
:1010500031F491E08F3F19F403C091E001C090E0BA
:1010600090FF09C049815A816B817C818D819E816D
:101070000E949A1005C0C9010E947C068111F2CF1E
:101080002B960FB6F894DEBF0FBECDBFDF91CF9188
:101090000895FC01808191810E94F50D0895CF9300
:1010A000882309F49CC0C82F8238C1F40E944F2ABB
:1010B00081FD95C069E380910201909103010E9436
:1010C000192B0E949B112FEF81EE94E0215080405C
:1010D0009040E1F700C0000069E319C0833801F5D2
:1010E0000E944F2A80FD7BC063E5809102019091B0
:1010F00003010E94192B0E949B112FEF81EE94E0B7
:10110000215080409040E1F700C0000063E58091ED
:101110000201909103010E941B2BCF910C949B1113
:101120008438C1F40E944F2A82FD59C067E480913F
:101130000201909103010E94192B0E949B112FEF35
:1011400081EE94E0215080409040E1F700C0000023
:1011500067E4DDCF8CEF8C0F813AD0F46C2F809157
:101160000201909103010E94E32A882349F06C2F29
:1011700080910201909103010E941B2B0E949B1100
:101180006C2F80910201909103010E94192BC5CF11
:1011900080E28C0F883048F4C77081E001C0880F6E
:1011A000CA95EAF70E945C11B8CFEBE5EC0FE3308B
:1011B00040F4F0E0ED58FE4F808190E0CF910C9428
:1011C000AB2AC85AC73158F4EC2FF0E0EE0FFF1FDE
:1011D000EB5BFE4F80819181CF910C94C12ACF911E
:1011E0000895882309F45BC0682F823879F40E943F
:1011F0004F2A81FF54C069E380910201909103015D
:101200000E94192B0E949B1169E310C08338B1F42E
:101210000E944F2A80FF43C063E5809102019091B4
:1012200003010E94192B0E949B1163E5809102012A
:10123000909103010E941B2B0C949B11843879F42C
:101240000E944F2A82FF2BC067E480910201909197
:1012500003010E94192B0E949B1167E4E7CF8CEFDA
:10126000860F813A18F380E2860F883048F4677061
:1012700081E001C0880F6A95EAF70E946211DCCF15
:101280008BE5860F833020F480E090E00C94AB2A4D
:10129000685A673120F480E090E00C94C12A0895E8
:1012A0001F93CF93DF93182FEB010E944F082097D5
:1012B00041F08FE99FE00197F1F700C0000021970E
:1012C000F6CF812FDF91CF911F910C94F1088933D4
:1012D00019F060E070E002C060E570E00C94500925
:1012E000882321F00E945C110C949B11089588239F
:1012F00021F00E9462110C949B110895CF92DF920D
:10130000EF92FF920F931F93CF93DF937C01D62F21
:10131000C72FFC011281058102950F700E945211A6
:101320008823B9F01123A9F08C2F807F803421F01D
:1013300080E28D0F883068F08091F30282FD09C051
:1013400082E00E94FB110E94521191E0D82ED92612
:1013500001C0D12CCC2EC2948FE0C8228C2D90E0FD
:101360008C30910508F0C4C1FC01EA5AFF4F0C947F
:101370002A348C2F807FCF70882311F0C295C07FD4
:10138000112399F0CC2309F49FC180E28D0F88309E
:1013900010F0D11104C08C2F0E945C1103C08C2F5F
:1013A0000E946C110E949B118FC18D2F0E94F10829
:1013B000CC2309F49DC180E28D0F883038F1DD2304
:1013C00029F18C2F0E94721124C08C2F807FCF7046
:1013D000803211F0C295C07FDD2319F0D130A1F128
:1013E0003DC08091F30282FF17C0112349F0CC2346
:1013F00029F08C2F0E945C110E949B1180E065C136
:1014000080E00E94F108CC2309F472C18C2F0E9465
:1014100062110E949B116CC1112371F0002341F0F5
:10142000013031F40E947C118C2B0E94841160C128
:101430000E947C118C2B1DC0002319F0013009F48F
:1014400057C10E94911125C0112321F0063008F0E8
:101450004FC10EC0053008F04BC11BC0112361F015
:10146000002331F0F701858180FF2EC18F708583C5
:101470008C2F0E9470093CC1002359F0D93309F028
:1014800034C1FFEF07EE13E0F15000401040E1F7E8
:101490002AC18C2F0E9477092BC18C2F86958695A7
:1014A000837019F0813061F023C1112321F08D2F59
:1014B0009C2F937002C080E090E00E94AB2A20C174
:1014C000112321F08D2F9C2F937002C080E090E0BB
:1014D0000E94C12A15C18C2F837009F047C01111D9
:1014E0000BC12D2F229526952770220F220F6D2FCD
:1014F0006F70862F90E0A0E0B0E0022E04C0880F4D
:10150000991FAA1FBB1F0A94D2F7D4FF10C04FE047
:1015100050E060E070E004C0440F551F661F771F65
:101520002A95D2F7409550956095709503C040E09C
:1015300050E0BA01C695C695C3708A019B01082B7D
:10154000192B2A2B3B2BC901B801C23049F058F4A2
:10155000C13019F00E94700CCFC00E945E0CCCC04C
:101560000E94820CC9C00E945C0CC6C0112319F0F5
:101570008C2F817001C08695882309F4BDC02D2F62
:10158000229526952770220F220F6D2F6F70862FC0
:1015900090E0A0E0B0E0022E04C0880F991FAA1FBF
:1015A000BB1F0A94D2F7D4FF10C04FE050E060E0B8
:1015B00070E004C0440F551F661F771F2A95D2F7AD
:1015C000409550956095709503C040E050E0BA0199
:1015D000C695C695C3708A019B01082B192B2A2B2F
:1015E0003B2BC901B801C23049F058F4C13019F0A1
:1015F0000E94350D81C00E94230D7EC00E94470DC0
:101600007BC00E94960C78C0CF70112339F08C2FCC
:101610000E94BC0C8D2F0E9470096EC08D2F0E94FD
:1016200077098C2F0E94DD0C67C0D23F21F128F48E
:10163000D03F41F0D13FC1F043C0D33F19F1D43F77
:1016400079F03EC0112341F0053008F051C08C2FD5
:101650008F710E94020D4CC0063008F049C0F7CFD0
:101660008091F30282FF18C0112339F08C2F8F7103
:101670000E94BC0C3DC01123C9F38C2F8F710E94B6
:10168000DD0C36C0112329F08C2F8F710E94A70C1E
:101690002FC00E94A20C2CC0112349F0CF718C2FB7
:1016A0000E94BC0C63E08C2F0E94E01121C081E0FD
:1016B0000E94FB110230E0F082E00E94FB1118C092
:1016C000112331F0002391F28D2F0E944F0810C09A
:1016D000002399F2D93349F41FEF27EE33E011507C
:1016E00020403040E1F700C000008D2F0E94F1083B
:1016F00088EF8C0D843020F40E944F2A0E94BD0791
:10170000DD20C9F00E944E1180FD15C0F701128244
:101710000E9448110E94BC0CC7010E94BC0B0E9491
:101720004811DF91CF911F910F91FF90EF90DF90C3
:10173000CF900C94DD0CDF91CF911F910F91FF9012
:10174000EF90DF90CF9008950F931F93CF93DF9387
:10175000EC01688179818A810E94000E8C010E94CF
:10176000590D0E944A0CB801CE010E947E09DF91FA
:10177000CF911F910F910895CF93DF93EC01988142
:1017800089812B813C81232B31F08F3F31F481E023
:101790009F3F19F403C081E001C080E080FD1DC0BF
:1017A000CE010E941D07811110C00E945211882392
:1017B000A1F08A81882389F08091F30282FD0DC017
:1017C00082E0DF91CF910C94FB11CE010E94A40B1B
:1017D000CE01DF91CF910C947E06DF91CF910895D9
:1017E00080E090E00E94AB2A80E090E00E94C12A55
:1017F0000E9479110C949B11809102019091030138
:101800000E941D2B0C94F00B0E9469110C94FC0B90
:1018100092959F70963079F010F4925001C09A50D2
:10182000923068F4803F69F018F4883E40F409C0B3
:10183000843F29F406C0883E20F0813F11F080E00B
:10184000089581E00895FC01808191810E94F50D49
:101850000E94080C0895CF93DF9300D000D01F9210
:10186000CDB7DEB70F900F900F900F900F90DF91D4
:10187000CF910895CF93DF9300D000D000D0CDB7A3
:10188000DEB726960FB6F894DEBF0FBECDBFDF9150
:10189000CF910895089508950C944B0C0C944C0C22
:1018A0000E944E0C60933A0270933B0280933C027C
:1018B00090933D020C94F00B0C94500C0F931F93DB
:1018C00000913A0210913B0220913C0230913D027E
:1018D000602B712B822B932B1F910F910C94500C2A
:1018E0000F931F9300913A0210913B0220913C020A
:1018F00030913D0260237123822393231F910F9126
:101900000C94500C0F931F9300913A0210913B02DC
:1019100020913C0230913D02602771278227932756
:101920001F910F910C94500C0C944B0C0E94940C32
:101930006093360270933702809338029093390295
:101940000C94F00B60E070E0CB010C94960C0F93BC
:101950001F9341E050E060E070E08A019B0104C009
:10196000000F111F221F331F8A95D2F7C901B8013A
:101970001F910F910C94960C0F931F9341E050E030
:1019800060E070E004C0440F551F661F771F8A9502
:10199000D2F78091360290913702A0913802B0912F
:1019A00039028A019B01082B192B2A2B3B2BC901D9
:1019B000B8011F910F910C94960C0F931F9341E067
:1019C00050E060E070E004C0440F551F661F771FB1
:1019D0008A95D2F740955095609570958091360222
:1019E00090913702A0913802B09139028A019B018F
:1019F000082319232A233B23C901B8011F910F9102
:101A00000C94960C0F931F9341E050E060E070E05F
:101A100004C0440F551F661F771F8A95D2F7809127
:101A2000360290913702A0913802B09139028A01B2
:101A30009B01082719272A273B27C901B8011F91B5
:101A40000F910C94960C0F931F93009136021091F6
:101A500037022091380230913902602B712B822B92
:101A6000932B1F910F910C94960C0F931F93009141
:101A700036021091370220913802309139026023EA
:101A80007123822393231F910F910C94960C0F9333
:101A90001F93009136021091370220913802309145
:101AA000390260277127822793271F910F910C9489
:101AB000960C0895292F220F920F990F890FE82F66
:101AC000E695E695E695877051E001C0550F8A9539
:101AD000EAF785E0E89FF0011124E25FFD4F20E086
:101AE00030E070E04081CB01022E02C096958795D0
:101AF0000A94E2F781708195842785238427819356
:101B00002F5F3F4F2530310569F70895292F220FA8
:101B1000920F990F890F682F669566956695982F95
:101B2000977085E0689FB001112440E050E080E0AC
:101B3000FB01E40FF51FE25FFD4F208130E0092E2D
:101B400002C0369527950A94E2F721703327042EB8
:101B500001C0220F0A94EAF7822B4F5F5F4F453096
:101B6000510531F70895BF92CF92DF92EF92FF9225
:101B70000F931F93CF93DF938C01C0903602D090C8
:101B80003702E0903802F090390280913A02909149
:101B90003B02A0913C02B0913D02C82AD92AEA2A10
:101BA000FB2ACFE1D0E0D701C6010C2E04C0B695C8
:101BB000A795979587950A94D2F780FD04C0219741
:101BC00090F7B12C07C0BC2EB8018C2F0E940415D1
:101BD0000197A9F38B2DDF91CF911F910F91FF906A
:101BE000EF90DF90CF90BF900895CF93DF93EC01FB
:101BF0000E94B30DBE010E940415DF91CF9108959C
:101C00001F93CF93DF93EB0190910D02992321F065
:101C1000CB010E94F50D13C0882349F0CB010E942F
:101C2000B30D182F682FCE010E945A0D04C0CB01AE
:101C30000E94860D182FBE01812F0E940415DF918E
:101C4000CF911F9108951F93CF93DF93C0913E02D0
:101C500016E080913F02C81799F0D0E01C9FF00178
:101C60001D9FF00D1124E05CFD4F40815181628188
:101C70007381848195810E943A0C2196C770E9CFC7
:101C8000DF91CF911F9108954091700250917102A0
:101C9000609172027091730280917402909175024A
:101CA0000C943A0CEF92FF920F931F93CF93DF9314
:101CB0008091750282958F7009F065C080917202E3
:101CC000882309F460C080913E02F0903F02109199
:101CD000700200917102609173027091740291E040
:101CE0001F3F09F090E0C0910001D0910101292F20
:101CF00096E0E92E8F1509F446C06115710521F0B3
:101D00000F3F21F030E003C031E001C0322F90E0FE
:101D100030FD36C0E89EF001E99EF00D1124DF0190
:101D2000A05CBD4F11963C911197301329C03C9196
:101D3000311326C012963C911297311121C013968F
:101D40004D915C911497461B570B4C175D07C0F4DF
:101D5000809175028F70806180937502EB5BFD4FFF
:101D600080818F708061808380E792E00E94BC0B4D
:101D7000DF91CF911F910F91FF90EF900C94230E64
:101D800001968770B7CFDF91CF911F910F91FF9090
:101D9000EF9008959F92AF92BF92CF92DF92EF9211
:101DA000FF920F931F93CF93DF93CDB7DEB7619769
:101DB0000FB6F894DEBF0FBECDBF8C0185E0F801F1
:101DC000DE011D9601900D928A95E1F7D8011296D9
:101DD000EC9090917002E091710220917302309129
:101DE00074022115310531F0EF3F31F481E09F3F5E
:101DF00019F403C081E001C080E0B82FB1709B2EC0
:101E000080FD47C1D8014C9111965C9111971396B2
:101E1000AD90BC90149780E7C82E82E0D82EF09049
:101E20007202B501621B730B209100013091010118
:101E3000FF2009F4D9C0809175026217730708F07A
:101E400095C0282F207F09F052C05E1313C049139C
:101E500011C0FE2CE1100EC08F708061809375025E
:101E60000E94440EC6010E94BC0B80917502F801CD
:101E700085834DC1AB2831F05F3F31F481E04F3FA6
:101E800019F403C081E001C080E080FD03C081E05F
:101E90008E2502C080E090E0F82FF170FF2E80FFC9
:101EA0001CC080913E0220913F0236E0821709F467
:101EB0000BC190E0389FF001399FF00D1124E05CD8
:101EC000FD4F6181561306C06081461303C06281D5
:101ED000E61203C001968770E9CFFE2CEE2009F4CC
:101EE00016C18091750281608093750254C05E13A3
:101EF00006C0491304C0E11002C0F80199C0C8012E
:101F00000E94230C882361F1EE2051F1209175028B
:101F1000822F82958F7090E0029774F0809170020A
:101F20009091710298878F831986BB86AA862C8729
:101F3000CE0107960E94BC0B86E0F801A0E7B2E054
:101F400001900D928A95E1F70E94520E0E94440E74
:101F50000AC05E1711F1C8010E94230C81112CC028
:101F6000C8010E94BC0BFF24F394D1C0282F207F0E
:101F700081F77A2DB98AA88A6E2D89890E942B0C47
:101F800080E792E00E94BC0B86E0D6011D928A9504
:101F9000E9F70E94440EF12CBAC04913DCCFE110DE
:101FA000DACFF8018583C8010E94BC0B86E0D60118
:101FB0001D928A95E9F7ABC0EE2091F2209175024F
:101FC000822F82958F7090E002970CF4B5CF8091AC
:101FD0007002909171029A8389831B82BD82AC82C8
:101FE0002E83CE010196A6CF6217730708F044C076
:101FF000FE2CEE2009F4B4CF5E1330C049132EC07E
:102000002091750220FD21C0822F82958F70482F6C
:1020100050E041155105C9F0F80125834F305105B5
:1020200041F08F5F982F9295907F822F8F70892B30
:102030008583C8010E94BC0B86E0F801A0E7B2E0EE
:1020400001900D928A95E1F73CC086E0F801A0E787
:10205000B2E001900D928A95E1F759C0C8010E9443
:10206000230C811169CF8091750281608093750284
:10207000C8010E94BC0B4BC07A2DB98AA88A6E2D6C
:1020800089890E942B0C86E0D6011D928A95E9F77A
:1020900018C0EE2009F464CFC8010E94230CF82E6A
:1020A000882309F45DCF86E0F801A0E7B2E0019053
:1020B0000D928A95E1F780E792E00E9449080E941C
:1020C000520E0E94440E23C04D875E878D859E85EB
:1020D0000E94F50D292F22952F70223028F49F7031
:1020E00039F0811105C00BC0243028F49F7049F4E9
:1020F000805E883020F0C8010E94BC0B9F2CF92C18
:1021000006C0D80115969C91907F91F7F8CF8F2D3E
:1021100061960FB6F894DEBF0FBECDBFDF91CF91B1
:102120001F910F91FF90EF90DF90CF90BF90AF90F5
:102130009F9008951F93CF93DF93CDB7DEB72C9771
:102140000FB6F894DEBF0FBECDBF4F8358876987A7
:102150007A878B879C87CE0107960E94CA0E8823B8
:10216000D1F09F8188852A853B85232B31F08F3FD5
:1021700031F481E09F3F19F403C081E001C080E0A9
:1021800080FD47C04F81588569857A858B859C8500
:102190000E943A0C3EC086E0FE013796DE011196A1
:1021A00001900D928A95E1F7FF81E8856A857B852C
:1021B0006115710531F0EF3F31F481E0FF3F19F413
:1021C00003C081E001C080E080FD23C020913F0278
:1021D00030E0C90101968770992740913E0250E096
:1021E00084179507F1F1F983EA837D836C8396E088
:1021F000929FD001939FB00D1124A05CBD4FFE01B2
:10220000319601900D929A95E1F780933F020E94DA
:10221000230E16E080913E0290913F02891771F1E2
:10222000189FC0011124805C9D4F0E94CA0E882314
:1022300029F1E0913E021E9FF0011124E05CFD4F68
:102240004081518162817381848195810E943A0C21
:1022500080913E0290E001968770992780933E021C
:10226000D9CF0E94040C10923F0210923E02E0E788
:10227000F2E086E0DF011D928A95E9F72C960FB611
:10228000F894DEBF0FBECDBFDF91CF911F910895AF
:1022900080917E02859585958595089580917E0231
:1022A0008770089590917E02977081E009F480E034
:1022B000089580918902089590918902892B8093D5
:1022C00089020895809590918902892380938902DB
:1022D000089510928902089590918802892B809325
:1022E00088020895809590918802892380938802BE
:1022F000089510928802089580917F0208950895AC
:102300000C947F110C9480119091F30292FD08C0FF
:1023100090917F02981721F080937F020C94821194
:10232000089580917F02882329F010927F0280E037
:102330000C9482110895CF93DF93E0910201F09104
:102340000301809189028083E0910201F0910301F1
:10235000908180918802892B808380917F028823DD
:1023600081F0E0910201F09103019081892B80833B
:1023700080910201909103010E94D72A81110E944D
:102380009111C0910201D091030148E050E066E74D
:1023900072E0CE010E946E34892B69F088E0FE0164
:1023A000A6E7B2E001900D928A95E1F7CE01DF91A8
:1023B000CF910C94622ADF91CF9108950C947F11F4
:1023C0009091F30292FD10C098E0899F9001112432
:1023D000262B20937E020E94BC0C80917E02859564
:1023E000859585950C94DE110C94BC0C10927E02A0
:1023F00080E00C94DE1120917E02809582238093F0
:102400007E02982F977099F430E0482F082E000C28
:10241000550B2417350759F09091F30292FD07C030
:102420008595859585950E94DD0C0C94F61108958F
:10243000CF939091F30292FB222720F92817F9F00D
:10244000C82F892FC0FB82F98093F3028091F2029A
:102450009091F3020E94791282E00E94FB11809118
:102460009C0280FF0CC01F92CF938DEE92E09F9351
:102470008F930E94F0050F900F900F900F90CF91C7
:1024800008958091F30282FB882780F991E08927E3
:102490000C94181281E00C94181280E00C9418121D
:1024A00080E090E00E94923421E0893E9E4F09F046
:1024B00020E0822F089582E090E00C94843483E041
:1024C00090E00C948434682F83E090E00C9498346E
:1024D000CF9384E090E00E948434C82F82E290E0A1
:1024E0000E9484342C2F30E0A901582BCA01CF91CF
:1024F0000895CF93C92F682F84E090E00E9498340C
:102500006C2F82E290E0CF910C949834AB01BC0127
:102510008FE090E00C94AA34AB01BC0183E190E021
:102520000C94AA3460E070E0CB010C948C1260E053
:1025300070E0CB010E9486120C94921269EE7EEF3D
:1025400080E090E00E94B63460E082E090E00E947B
:10255000983460E083E090E00E94983410923A0250
:1025600010923B0210923C0210923D0260E084E027
:1025700090E00E94983460E082E290E00E949834FB
:1025800060E085E090E00E94983460E086E090E0B2
:102590000E9498346FEF87E090E00E94983440E00A
:1025A00050E0BA0188E090E00E94AA3460E08DE03B
:1025B00090E00E94983440E050E0BA0188E190E059
:1025C0000E94AA3460E087E190E00E94983440E0E5
:1025D00050E0BA018CE190E00E94AA3460E070E023
:1025E00080E290E00E94B63440E050E0BA0188E119
:1025F00090E00E94AA340C9497120C949E128EE0E4
:1026000090E00E94843491E0811101C090E0892F14
:102610000895682F8EE090E00C9498340E94CB2BA4
:10262000609398027093990280939A0290939B0210
:102630006093940270939502809396029093970210
:10264000089585B7806885BF85B7806885BF089580
:102650000C94601808950C942A130C942A130C946B
:102660002D130C942A130C9431130C942A130E94EA
:1026700021138EEE9DE20E94452A0E9435130C9490
:1026800033130E942B130C942A130E942B160E94C2
:10269000BC070C94F2250E94B62B0E94E0150E9404
:1026A00078180E94AF170E9445130E942D260E94A1
:1026B000BF230E9478210E9482180C942F138F92BE
:1026C0009F92AF92BF92CF92DF92EF92FF920F93C1
:1026D0001F93CF93DF93CDB7DEB72A970FB6F89449
:1026E000DEBF0FBECDBF0E94D317982E81110E946E
:1026F0000E138AE8A82E82E0B82E00E010E0802EAB
:10270000802F0E944F16D82EF501C1905F01C82678
:10271000B1F40F5F1F4F0A30110589F78FEF8983DE
:102720008A831B820E94BF2B8160782F9D838C83BC
:1027300049815A816B818D810E94FF072FC0809152
:102740009C0281FD0E945516E12CFF24F3948C2DF0
:102750008F21F1F00E942813882399F0EE828F8256
:10276000DF2081E009F480E088870E94BF2B816030
:10277000782F9A8789874E815F8168858A850E9434
:10278000FF07F801E657FD4F8081F826F08206C06A
:10279000E394FF0CF6E0EF12DACFBBCF81E09110AB
:1027A00001C080E02A960FB6F894DEBF0FBECDBF01
:1027B000DF91CF911F910F91FF90EF90DF90CF901D
:1027C000BF90AF909F908F9008950E945F130E94DA
:1027D00060180E9427220E94F1250C94CD07CF9308
:1027E000DF930E940915EC01811522E59207E8F5B7
:1027F000811531E5930708F0B6C0883E910528F5AC
:10280000803E910508F0E9C0883A910570F4853A58
:10281000910508F07AC08130910509F473C008F47D
:10282000D9C0049708F0D9C0D5C08F3B910508F0F6
:10283000D1C0C85AD0E0CC0FDD1FCA58DE4F099076
:10284000D881C02DCE019464C9C0811540E594079C
:1028500008F069C0811550E4950708F060C09A95AA
:1028600081159F4108F4B9C0B5C0811536E59307BD
:1028700028F5811545E5940708F092C0811554E5C7
:10288000950708F087C0AC0143705527282F26957F
:102890002695C115D34508F06CC081E090E002C0D8
:1028A000880F991F4A95E2F740E2249F9001112476
:1028B000EC01C22BD32BCE019C6890C081152AE578
:1028C000920780F4811539E5930708F072C08115ED
:1028D00048E5940708F47EC0D82FCC27CE01806F3E
:1028E000906A7CC090568115904208F073C08D2F7D
:1028F0008F710E949D15DD27D0628F71AE01582B1C
:10290000CA016CC081E090E069C0C55AD0E0CC55E6
:10291000DE4F8881C82FD0E0CE0190645FC0DF70A9
:10292000CE01906A5BC074E0969587957A95E1F741
:10293000282F23703C2F337081E090E002C0880F75
:10294000991F3A95E2F79C68AC01522B9A019C2F93
:102950009F709695969550E2959FE0011124C901CC
:102960008C2B9D2B3BC0D82FCC27CE01816F906A3A
:1029700035C081E090E002C0880F991F4A95E2F7C8
:1029800050E2259F90011124EC01C22BD32BCE01E4
:102990009A6824C0D82FCC27CE01846F906A1EC0BD
:1029A0000E949D158F7190E0D82FCC27CE019062A8
:1029B00015C08F700E949D1594E0D695C7959A9585
:1029C000E1F7CF70D0E0DC2FCC27D0699E01282B17
:1029D000C90104C080E090E001C0CE01DF91CF9139
:1029E00008952CE3829FC0011124FC0126E0729F10
:1029F000E00DF11D1124E60FF11DEE0FFF1FE8524F
:102A0000FF4F8591949108950E94F1140E94EF1355
:102A100008958238910569F1B0F48133910509F484
:102A20006DC048F48932910509F463C08A3291057A
:102A300009F469C008958533910509F455C08933B7
:102A40009105B9F00895833E910569F138F4803E0F
:102A50009105B1F0823E910509F10895863E9105F8
:102A6000A9F1873E9105B9F1843E910509F064C052
:102A700023C02091F20220FD4FC021FD4DC00895DA
:102A80008091F20280FD44C08091F30280FF44C037
:102A90008091F20284FD42C083EE4DC08091F2022B
:102AA00082FF38C0F5CF8091F20282FD33C0809161
:102AB000F30280FD31C0ECCF8091F30281FF32C080
:102AC0008091F20284FD2AC087EE35C08091F20227
:102AD00083FF26C0F5CF8091F20283FD21C0809153
:102AE000F30281FD1FC0ECCF8091F20285FD1CC076
:102AF0001DC08091F20285FD19C016C08091F202BE
:102B000086FD16C017C08091F20286FD13C010C06A
:102B100089E311C082EE0FC080EE0DC080E00BC0D3
:102B200086EE09C084EE07C089E205C085E303C0D4
:102B30008AE201C081E390E008959091F20292FF51
:102B40000DC0282F2871283019F4877F846006C0B3
:102B5000282F2471243011F48B7F886093FF0DC0DF
:102B6000282F2871283119F4877E846106C0282F08
:102B70002471243111F48B7E88612091F30220FFAF
:102B80000DC0382F3871383019F4877F816006C046
:102B9000382F3171313011F48E7F886021FF0DC0E4
:102BA000282F2871283119F4877E816106C0282FCB
:102BB0002171213111F48E7E886194FD877E089504
:102BC0001092EE021092EF021092F0021092F102B7
:102BD0000895CF92DF92EF92FF926B017C010E94E9
:102BE000601881110EC00E94CB2BC61AD70AE80AC2
:102BF000F90AC092EE02D092EF02E092F002F09257
:102C0000F102FF90EF90DF90CF9008950F931F9304
:102C10000E946018882321F01F910F910C94CB2BF8
:102C20000E94CB2B0091EE021091EF022091F00256
:102C30003091F102600F711F821F931F1F910F913E
:102C400008950E94601881110C94BF2B0E940616F3
:102C5000CB01089508950E945012811102C00E9474
:102C6000FD120E945B1280939C020E946812909356
:102C7000F3028093F2020E942A160E945F12682FCC
:102C800070E080E090E00E945C0C609136027091F0
:102C9000370280913802909139020C94940CE82FFD
:102CA000F0E0E150FD4F80810895CF92DF92EF92E6
:102CB000FF920F931F93CF93DF9381E193E00E94E4
:102CC00057058FEFE82E82E0F82EC0E0D0E09CE0C0
:102CD000C92E93E0D92E04E013E0DF93CF93DF9267
:102CE000CF920E94F00589E093E00E945705F7011A
:102CF00081917F010E94A3071F928F931F930F93CF
:102D00000E94F00582E093E00E94570521968DB75E
:102D10009EB708960FB6F8949EBF0FBE8DBFCA30FF
:102D2000D105D9F6DF91CF911F910F91FF90EF90D0
:102D3000DF90CF90089580EA8A95F1F7089500C05A
:102D400008950C949B1608950C94A3160C94A41645
:102D50000C94A3160C94A8160C94A316FF920F9330
:102D60001F93CF93DF9300D000D01F92CDB7DEB773
:102D70000E946018609109038823E9F185E0F82E2C
:102D80008E010F5F1F4FF8018F2D11928A95E9F781
:102D9000862F90E0B80181509D4F0E9490188823A3
:102DA00089F08091F40290E045E050E0B801815054
:102DB0009D4F0E946E3421E020939D02892B61F487
:102DC00010E016C080919D028823D1F3F801119282
:102DD000FA94E9F710929D02A091F402B0E0A1509C
:102DE000BD4F85E0F80101900D928A95E1F711E061
:102DF0000E940B070DC070E061507D4F8091F4027E
:102E000090E081509D4F0E942C190E94AC1610E05A
:102E1000812F0F900F900F900F900F90DF91CF9117
:102E20001F910F91FF900895F894E82FE295EF70AD
:102E3000F0E031A1282F2F7081E090E001C0880FD1
:102E40002A95EAF7982F9095932391A392A1892B25
:102E500082A3789408950F931F93CF93DF93CDEAC5
:102E6000D1E089918F3F11F00E94141781E0C23B9D
:102E7000D807B9F7C7EAD1E00DEA11E089918F3F91
:102E800011F00E9414170C171D07C1F7DF91CF91A5
:102E90001F910F910895CF92DF92EF92FF920F93BF
:102EA0001F93CF93DF938C01C62FD0E0CE018355C3
:102EB0009E4F7C01FC0190819F3F09F447C0D62EB4
:102EC000F894E92FE295EF70F0E081A19F7021E086
:102ED00030E001C0220F9A95EAF7822B81A382A1EC
:102EE0002095282322A378940E949F16E7EAF1E018
:102EF0004DEA51E031E0C12C21912F3F89F0A22F02
:102F0000A295AF70B0E090968C9190E02F7002C0C7
:102F1000959587952A95E2F780FD02C0832F01C021
:102F200080E0C82A330F4E175F0731F7F701808121
:102F30008F3F11F00E94141761E0C11001C060E0E2
:102F40008D2D0E94A116C00FD11FC882DF91CF9195
:102F50001F910F91FF90EF90DF90CF900895809197
:102F6000040180910401811102C095E001C090E04C
:102F70009093090385E0891B8093F4020E942B172C
:102F80008AE0EFEFF2E0DF01982F1D929A95E9F7C2
:102F9000E5EFF2E0DF011D928A95E9F785E00E94F6
:102FA00027180C940907EF92FF920F931F93CF936A
:102FB000DF93CDB7DEB72A970FB6F894DEBF0FBE0A
:102FC000CDBF8E010F5F1F4F8AE0F80111928A95E5
:102FD000E9F7F12C6F2DC8010E944B17F394F5E02F
:102FE000FF12F8CF4AE050E0B80185EF92E00E946E
:102FF0006E347C0121E0892B09F420E0E114F10416
:1030000041F08AE0F801A5EFB2E001900D928A95B7
:10301000E1F76091090370E061507D4F45E085EF75
:1030200092E00E942818EF2819F40E94AE1602C000
:1030300081E090E02A960FB6F894DEBF0FBECDBFB8
:10304000DF91CF911F910F91FF90EF900895089518
:10305000FF920F931F93CF93DF938C01F62ED72F00
:10306000C42F222349F081E08093A0020E94BF2B4D
:1030700090939F0280939E028091A0028823C1F0CA
:1030800080919E0290919F020E94D72B059780F01D
:10309000EF2DFD2FD8014C2F50E0CD01801B910B5F
:1030A000841795071CF48D918193F7CF1092A0029D
:1030B000DF91CF911F910F91FF9008950C94FF1213
:1030C0008091A30281110DC00E94A933811102C019
:1030D00082E001C081E08093A302823011F40E945B
:1030E000A43381E09091A302913009F080E008952B
:1030F0000E945E18809304010E94601881110C9454
:10310000DA1808950E946018811102C00C94DC182E
:10311000089581E09091A4029A3008F080E008952B
:10312000EF92FF920F931F93CF938C017B01C0917D
:10313000A402CA3038F4B701C8010E942A198111CB
:1031400026C00AC08091A1029091A2020E94D72BB2
:10315000843F914080F719C08091A4028F3F19F0FD
:103160008F5F8093A4028091A4028A30E0F00E94D5
:10317000BF2B9093A2028093A10280919C0280FFBA
:1031800004C083E393E00E94570580E00DC0CA307D
:1031900040F080919C0280FF04C080E293E00E9496
:1031A00057051092A40281E0CF911F910F91FF90DB
:1031B000EF9008950C94DE280C94E128DF92EF92B2
:1031C000FF920F931F93CF93DF937901C82F880F3E
:1031D000DD0B41155105A9F0FE0193E0EE0FFF1F35
:1031E0009A95E1F7EB5FFE4F818192818B559D4F60
:1031F000208130E04217530708F49A01A9010E9488
:103200007B34CE010E94CA29D82E8823D1F0011523
:103210001105B9F083E0CC0FDD1F8A95E1F7FE01BF
:10322000EB5FFE4F438150E00417150708F4A80137
:10323000CB5FDE4F6C817D816B557D4FC7010E9456
:103240007B348D2DDF91CF911F910F91FF90EF90E7
:10325000DF9008950C94A91A0C94D31A0F931F931E
:10326000CF93DF9300D000D0CDB7DEB76091BD0221
:103270007091BE028091BF029091C0020E94E62B25
:10328000643671058105910528F10E940616DC015E
:10329000CB010296A11DB11D89839A83AB83BC83A8
:1032A00000E010E020E030E044E050E0BE016F5F5D
:1032B0007F4F82E00E94DE18182F882361F00E9461
:1032C000CB2B6093BD027093BE028093BF0290939C
:1032D000C00201C011E0812F0F900F900F900F904E
:1032E000DF91CF911F910F9108958F929F92AF928E
:1032F000BF92CF92DF92EF92FF920F931F93CF93E3
:10330000DF937C015B01942E852E69010E94891850
:10331000811103C001E010E002C00AE010E0C1E04A
:10332000D0E0F894B501C701F601099578948111B0
:1033300029C021960C171D078CF0CC9F9001CD9FC2
:10334000300D300D112480E090E045E34A95F1F70F
:103350000000019628173907C1F7E3CF90919C022E
:10336000892F817090FF0FC08F929F9289E693E022
:103370009F938F930E94F0050F900F900F900F90E6
:1033800080E001C081E0DF91CF911F910F91FF900C
:10339000EF90DF90CF90BF90AF909F908F90089567
:1033A0000F931F93CF93DF931F92CDB7DEB70E9489
:1033B000A423882321F00E94B923182F01C010E014
:1033C0001983E091B201F091B30102856091C102CD
:1033D0007091C2028091C3029091C4020E94E62BB8
:1033E000643671058105910510F41017D1F000E0E5
:1033F00010E020E030E041E050E0BE016F5F7F4F21
:1034000083E00E94DE18182F882361F00E94CB2BE6
:103410006093C1027093C2028093C3029093C4026E
:1034200001C011E0812F0F90DF91CF911F910F917B
:103430000895AF92BF92CF92DF92EF92FF920F93D7
:103440001F93CF93DF9300D000D000D0CDB7DEB76D
:103450007B01C090B201D090B30101E010E09E0169
:103460002A5F3F4F40E050E060E070E080E00E9463
:10347000DE18182F882309F43EC056018FEFA81AD2
:10348000B80A6091B9027091BA028091BB02909122
:10349000BC020E94E62B643671058105910518F186
:1034A00005E010E09E012F5F3F4F40E050E060E0FC
:1034B00070E081E00E94DE18182F65E070E0C50121
:1034C0000E942E2691E02E81281390E0192339F1D5
:1034D0000E94CB2B6093B9027093BA028093BB0217
:1034E0009093BC0211C065E070E0C5010E942E26D9
:1034F0009E818913D5CF85E0F6013196DE011196C4
:1035000001900D928A95E1F7112349F085E0FE01C3
:103510003196A4EBB2E001900D928A95E1F785E037
:10352000E4EBF2E0D70101900D928A95E1F7812F4B
:1035300026960FB6F894DEBF0FBECDBFDF91CF91B8
:103540001F910F91FF90EF90DF90CF90BF90AF90C1
:1035500008950F931F93CF93DF93EC018B0129E123
:103560003AE144EB51E00E9475198823B1F02EE254
:1035700039E141EC51E0B801CE010E947519882370
:1035800061F020ED39E14CEC51E0B801CE01DF9162
:10359000CF911F910F910C94751980E0DF91CF911D
:1035A0001F910F9108950F931F93CF93DF93F8947A
:1035B000C091B201D091B301CE01019625E0FB018B
:1035C000DC0101900D922A95E1F765E070E00E9420
:1035D0002E2688837894F8946E817F8188859985DA
:1035E0000091B0021091B1022091B2023091B30269
:1035F000601771078207930751F06093B0027093D0
:10360000B1028093B2029093B3020E94E9157894BC
:10361000F8948A850E943C257894DF91CF911F9180
:103620000F9108950E946A2E0E944B130C94762EDF
:103630000E947A2E0E94E5130C94982E0E945D2B16
:103640000E94512E0E9437130E94121B0E94181BC9
:103650000E944113FBCFEF92FF920F931F93CF93E2
:10366000DF938B01682F11110AC0442329F0E82F42
:10367000F0E0ED50F84F6491762F862F75C0212F22
:1036800030E0E82FF0E0442321F0ED50F84FE491D2
:10369000F0E046E0049FC0011124CFEFD0E0BE016E
:1036A0000E94E0334BEA4603C001479F900D11246E
:1036B000800F911D800F911D982F990F890FAE01DA
:1036C000421B530B4E9FD0014F9FB00D5E9FB00D1C
:1036D00011249B2F189FA0011124452F55278E01DF
:1036E000041B150B0E9FA0010F9F500D1E9F500D28
:1036F00011247E01E81AF108E29E8001E39E100D7C
:10370000F29E100D1124212F3327C21BD30BCE9F05
:103710009001CF9F300DDE9F300D11246230710576
:10372000A9F048F46115710569F061307105C9F4BB
:103730008B2F752F0DC06430710581F058F0663005
:10374000710579F47E2F8B2F932F0DC0832F7B2F44
:103750009E2F09C08E2F7B2F952F05C08E2F732F84
:1037600002C07E2F852F692FDF91CF911F910F917E
:10377000FF90EF90089541E00E942B1B089508955B
:103780000E94BB1B0895CF93DF93762FE901682F2A
:10379000842F0E94C01B798368838A83DF91CF9135
:1037A000089580910A03282F269530E021153105D0
:1037B00019F48170826005C02532310524F08170D2
:1037C000886480930A03089588E090E00C948C3418
:1037D000CF92DF92EF92FF926B017C010E94D11B8E
:1037E000B701A60188E090E0FF90EF90DF90CF90C6
:1037F0000C94AA34EAE0F3E083E0808311828FEF37
:1038000082838383148260817181828193810C948D
:10381000E81B80919C0280FF08C084E496E09F939F
:103820008F930E94F0050F900F9080919C0280FF73
:103830000FC080910A0381701F928F9387E296E0F8
:103840009F938F930E94F0050F900F900F900F9011
:1038500080919C0280FF0FC080910A0386951F9281
:103860008F938CE096E09F938F930E94F0050F90CA
:103870000F900F900F9080919C0280FF0EC080915E
:103880000B031F928F9382EF95E09F938F930E947B
:10389000F0050F900F900F900F9080919C0280FF89
:1038A0000EC080910C031F928F9388ED95E09F933B
:1038B0008F930E94F0050F900F900F900F908091C2
:1038C0009C0280FF0EC080910D031F928F938EEBA0
:1038D00095E09F938F930E94F0050F900F900F90AB
:1038E0000F9080919C0280FF0EC080910E031F926A
:1038F0008F9382EA95E09F938F930E94F0050F903B
:103900000F900F900F90089580910A0380FF02C0DE
:103910008695089580E0089590910E03933018F4F1
:103920009F5F90930E03882351F060910A0370917A
:103930000B0380910C0390910D030C94E81B0895E8
:1039400081E00C948C1C90910E03992319F09150F6
:1039500090930E03882351F060910A0370910B033A
:1039600080910C0390910D030C94E81B089581E065
:103970000C94A31C70E00C940226609129018091A4
:103980000A0380FF0AC08091280123E0829FC001C2
:103990001124815F9C4F0C94BA1C80912A01909154
:1039A0002B01891780F7E82FF0E09F01220F331FCA
:1039B000E20FF31FE15FFC4F1182108212828F5FD2
:1039C000F0CF90910A0390FF16C090912A012091A8
:1039D0002B01921770F4E92FF0E0DF01AA0FBB1F53
:1039E000EA0FFB1FE15FFC4F8183608342839F5F8F
:1039F000F0CF0C94BD1C0895CF93DF9300D01F929D
:103A0000CDB7DEB790910A0390FF0AC09E012F5FE9
:103A10003F4F0E94C31B4B8169818A810E94E11C38
:103A20000F900F900F90DF91CF910895CF93DF9378
:103A3000EC01EC81F0E0E159F94F4491EAE0F3E068
:103A4000628181810E94FC1C8C818F5F8C83DF915D
:103A5000CF910895CF93DF93EC01EAE0F3E0438147
:103A600062818C810E94FC1C8C818F5F8C83DF9132
:103A7000CF9108950F931F93CF93DF9300D01F92A0
:103A8000CDB7DEB78C018091C50281110AC09E01BD
:103A90002F5F3F4F4FEF6FEF0E94C31B8A818093D0
:103AA000C502F8018481813051F028F0823061F440
:103AB0004091C5020AC08091C50240E007C06091F4
:103AC000C50240E080E003C040E080E060E00E948A
:103AD000E11CF801848190E0019663E070E00E94AF
:103AE000F43384830F900F900F90DF91CF911F914B
:103AF0000F9108954F925F926F927F928F929F9253
:103B0000AF92BF92CF92DF92EF92FF920F931F93EB
:103B1000CF93DF9300D01F92CDB7DEB7F82EB62E2D
:103B2000E42E622E90910A0390FFB4C0E92FE6952F
:103B3000AE2FB0E0AA52BE4F8C918093CF029E7FF1
:103B4000923061F49E012F5F3F4F8F2D0E94C31B67
:103B50004B8169818A810E94E11C62C0823019F424
:103B6000E0900D035DC0863019F4F0900B0358C04F
:103B70008930D9F3893109F053C0E9518E2F817012
:103B8000782E81E0A72CA826E695F0E0E159F84FC1
:103B9000C590D490412CDD249DEF892E93E0992E81
:103BA00060912C014616D0F5042D10E00C9DC0014B
:103BB0000D9D900D1C9D900D112470E00E94E0332E
:103BC0005F2C711002C0560E01C0561A80919C02E3
:103BD00080FF11C0DF92CF921F92AF921F925F922F
:103BE0001F924F929F928F920E94F0050FB6F89409
:103BF000DEBF0FBECDBF80912A01080F111D9801B5
:103C0000220F331F020F131F9801215F3C4F4E2DCF
:103C10006B2D852D0E94C31B4394C2CF0E94BD1CF7
:103C2000F0920B03B0920C03E0920D036620E9F0D2
:103C300060910A0370910B0380910C0390910D0326
:103C40000E94E81B80919C0280FF24C080910D039C
:103C50001F928F9380910C031F928F9380910B037F
:103C60001F928F9388ED93E00CC080919C0280FF9F
:103C700011C01F92EF921F92BF921F92FF9281EB91
:103C800093E09F938F930E94F0050FB6F894DEBFE8
:103C90000FBECDBF0F900F900F90DF91CF911F916E
:103CA0000F91FF90EF90DF90CF90BF90AF909F90DB
:103CB0008F907F906F905F904F900895EAE0F3E0CF
:103CC0009181282F4381628188E0890F0C947A1DAD
:103CD00081E00C945E1EEAE0F3E09181282F43819D
:103CE000628188EF890F0C947A1D81E00C946B1E21
:103CF000EAE0F3E0628121E1620F08F46FEF282F20
:103D0000438181810C947A1D81E00C94781EEAE055
:103D1000F3E0628121E1621B08F460E0282F438117
:103D200081810C947A1D81E00C94871EEAE0F3E017
:103D3000438121E1420F08F44FEF282F62818181F6
:103D40000C947A1D81E00C94961EEAE0F3E0438126
:103D500021E1421B08F440E0282F628181810C940C
:103D60007A1D81E00C94A51E20E00C947A1DFF9230
:103D70000F931F93CF93DF93EC01F12C0FEF10E023
:103D800060912C01F616F0F480912A012F2D30E07D
:103D9000280F311DC901880F991F280F391F215F76
:103DA0003C4F70E0C8010E94F433962F8C81409103
:103DB0000D0360910C03F99E800D11240E94C31B1A
:103DC000F394DECF0E94BD1C9A818C8190FF02C0CB
:103DD0008F5F01C081508C83DF91CF911F910F9134
:103DE000FF900895AF92BF92CF92DF92EF92FF9231
:103DF0000F931F93CF93DF93FC01828180FF02C05A
:103E00000FEF01C001E010E04CE0A42E80912C01E6
:103E1000181708F043C080912A01C12ED12CE60169
:103E2000C80FD11DCE01880F991FC80FD91FC15FC0
:103E3000DC4F198218821A8234E0E32EF12CB12C67
:103E40008091C7028B0D8D302CF06A2D0E94D233E9
:103E5000892F05C087FF03C090912C01890F082E80
:103E6000000C990BC816D90691F480910D038E9D14
:103E7000A0018F9D500D1124559547955595479557
:103E80009E0160910C0380910B030E94C31BB00E36
:103E9000F1E0EF1AF108A1F61F5FB8CF0E94BD1C38
:103EA0008091C702013031F4811102C080912C0150
:103EB000815007C090E0019660912C0170E00E9453
:103EC000F4338093C702DF91CF911F910F91FF9040
:103ED000EF90DF90CF90BF90AF900895CF938091F7
:103EE0002A0190912B01891770F4E82FF0E09F01CF
:103EF000220F331FE20FF31FE15FFC4F118210828C
:103F000012828F5FF0CFC0E060912C01C617C0F520
:103F1000EC2FF0E070E0CF010E94F43320912A01F1
:103F2000820F2091C602022E000C330B90E0E217A4
:103F3000F307CCF020912701022E000C330B2E1733
:103F40003F078CF09C01220F331F820F931F9C01AF
:103F5000215F3C4F40910D0360910C0380910B0356
:103F60000E94C31B0BC0FC01EE0FFF1F8E0F9F1F93
:103F7000FC01E15FFC4F118210821282CF5FC4CF3F
:103F80000E94BD1C209126018091C602820F809361
:103F9000C60290912701920F9093270119165CF4A5
:103FA000082E000C990B40912C0150E04150510912
:103FB000841795071CF0219520932601CF91089531
:103FC0008F929F92AF92BF92CF92DF92EF92FF9229
:103FD0000F931F93CF93DF938C01FC014481C42F77
:103FE000D0E09E01DE010E9438349B01AC010E94AA
:103FF0004E346B017C01E0E2F0E0EC1BFD0BA5E52B
:10400000B0E09B01AC010E944E344B015C019F016A
:10401000DF010E9430349B01AC010E9459349B01A6
:10402000AC012C0D3D1D4E1D5F1DC501B4010E944C
:104030000834C22FD22F2A3228F4F3E02F9F9001A8
:1040400011240DC025E530E02C1B3109C901880F72
:10405000991F280F391F37FF02C02F5F3F4F35953B
:104060002795C22FC095F12C85E5E82EED1A809199
:104070002C01F816C8F4F1FC02C08E2D01C08D2F62
:1040800090912A012F2D30E0290F311DA901440FF5
:10409000551F240F351F215F3C4F4C2F60910C039F
:1040A0000E94C31BF394E3CF0E94BD1CF8018481DE
:1040B000811102C091E003C0803219F49FEF909308
:1040C000250190912501890FF8018483DF91CF911B
:1040D0001F910F91FF90EF90DF90CF90BF90AF9026
:1040E0009F908F9008950F931F93CF93DF93EC01D0
:1040F00000E010E080912C01282F30E00217130718
:1041000024F590912A019801290F311DA901440F2E
:10411000551F240F351F215F3C4F869590E04C8141
:10412000081719071CF4442331F002C0411103C0E1
:1041300040910D0301C040E060910C0380910B039E
:104140000E94C31B0F5F1F4FD5CF0E94BD1C8C81E7
:1041500090E00196817099278C83DF91CF911F9118
:104160000F91089560910A03669570E04BE050E06E
:104170008DE291E00E946134892B19F481E08093F3
:10418000D0020E9421169093C9028093C8028091A8
:104190009C0280FF08C088E993E09F938F930E9460
:1041A000F0050F900F9008951092D00280919C021C
:1041B00080FF08C08FE793E09F938F930E94F005E4
:1041C0000F900F90089590910A0390FF54C0917042
:1041D000811102C0926006C0853210F0986402C05E
:1041E000880F982B90930A036623B1F060910A031D
:1041F00070910B0380910C0390910D030E94E81BBA
:1042000080919C0280FF1BC080910A0386951F92BB
:104210008F9388EE94E00BC080919C0280FF0FC0CA
:1042200080910A0386951F928F938AEC94E09F9366
:104230008F930E94F0050F900F900F900F90609158
:104240000A03669570E04BE050E08DE291E00E9439
:104250006134892B19F00E94D42002C00E94B22040
:1042600081E08093CB0240910D0360910C0380911B
:104270000B030C94B41E0895682F90910A03969531
:1042800081E0890F853208F081E00C94E32081E021
:104290000C943C21682F90910A0396958FEF890F1B
:1042A00009F484E20C94E32081E00C944A2161E05B
:1042B0000C94E32080910A03816080930A0380912B
:1042C0009C0280FF0DC01F9281E08F938CE594E0EB
:1042D0009F938F930E94F0050F900F900F900F9077
:1042E00080910A0386950C94572160E00C94E3209A
:1042F0008091CE02811160C080919C0280FF08C035
:104300008BE895E09F938F930E94F0050F900F909C
:1043100080919C0280FF08C085E795E09F938F9372
:104320000E94F0050F900F900E945012811110C052
:1043300080919C0280FF08C08DE495E09F938F934D
:104340000E94F0050F900F900E94FD120E94FA1B30
:104350000E94E41B60930A0370930B0380930C0389
:1043600090930D036E7FC1F480919C0280FF08C082
:1043700084E095E09F938F930E94F0050F900F903B
:104380000E94FA1B0E94E41B60930A0370930B03C4
:1043900080930C0390930D030E94D11B0E94091C73
:1043A0001092D00280910A0380FF03C086950E947C
:1043B000752181E08093CE02089580910A038E7F5B
:1043C00080930A0360910A0370910B0380910C03A0
:1043D00090910D030E94E81B80919C0280FF0FC00A
:1043E00080910A0381701F928F9384E294E09F93DF
:1043F0008F930E94F0050F900F900F900F900E94E6
:10440000D4202FEF80E792E0215080409040E1F7E8
:1044100000C000000C94BD1C80919C0280FF10C065
:1044200080910A03809581701F928F9383E994E0B5
:104430009F938F930E94F0050F900F900F900F9015
:1044400080910A0380FD0C94DD210C945A210F9376
:104450001F93CF93DF938091D002882309F485C006
:104460008091CF02E0910A03E695E81BE093CA022F
:10447000823049F4F0E0E559F94FE491CE2FD0E0D5
:1044800006E11DE149C0863049F4F0E0E859F94FF2
:10449000E491CE2FD0E00AE21DE13EC0893051F414
:1044A000E695F0E0EB59F94FE491CE2FD0E007EB21
:1044B0001EE132C08F3051F4E695F0E0EE59F94F2D
:1044C000E491CE2FD0E002EF1EE126C0853149F401
:1044D000F0E0E15AF94FE491CE2FD0E00EE61FE173
:1044E0001BC0883181F0833239F4EDE5F6E0C591E7
:1044F000D4910AE31DE110C0843251F4C4EFD1E03D
:1045000003E710E209C0C8E2D0E000EE1FE104C0FA
:10451000C0EDD7E00FEB1BE18091CB02882361F067
:104520001092CB020E9421169093C9028093C80278
:104530001092CD021092CC020E942116E091C80286
:10454000F091C9028E1B9F0B8F3F9F4770F4EC0FB9
:10455000FD1FF093C902E093C80288EC92E0F801D5
:10456000DF91CF911F910F910994DF91CF911F910E
:104570000F910895882311F0FA0101C0FB010994FD
:10458000CF93DF93C82FD62F0E94841C8C1740F046
:104590000E94841C8D1720F4DF91CF910C94472149
:1045A0008C2FDF91CF910C9457211F93CF93DF93E2
:1045B000FB0112811111C3C0EC010E9459118272DA
:1045C000CD3CFCE5DF0709F49AC0A8F5C73CECE553
:1045D000DE0709F476C0A8F4C43C9CE5D90709F4C9
:1045E0005FC028F4C33CDC4509F457C054C0C53C47
:1045F0009CE5D90709F459C0C63CDC4509F45CC008
:104600004AC0CA3CFCE5DF0709F46AC050F4C83C64
:10461000ECE5DE0709F45AC0C93CDC4509F45BC08F
:104620003AC0CB3C9CE5D90709F45FC0CC3CDC45E3
:1046300009F460C030C0C23DFCE5DF0709F46FC07B
:1046400088F4CF3C9CE5D90709F460C008F45CC04D
:10465000C03DFCE5DF0709F45CC0C13DDC4509F461
:104660005BC019C0C53D9CE5D90709F460C050F492
:10467000C33DFCE5DF0709F455C0C43DDC4509F442
:1046800054C009C0C63D9CE5D90709F455C0CE35D4
:10469000DD4509F454C011E052C00E940C224FC005
:1046A00044E551E267E471E204C047E451E264E5A5
:1046B00071E20E94BA2243C045E75EE168E67EE10E
:1046C000F8CF48E65EE165E77EE1F3CF43E95EE1DE
:1046D00064E87EE1EECF44E85EE163E97EE1E9CFA4
:1046E00041EB5EE162EA7EE1E4CF42EA5EE161EB4A
:1046F0007EE1DFCF47EB5CE160EA7CE1DACF40EAC4
:104700005CE167EB7CE1D5CF81E017C065E082E03A
:1047100010C068E086E00DC06EE089E00AC064E188
:104720008FE007C067E185E104C088E106C062E26E
:1047300089E10E94C02203C083E20E945721812F99
:10474000DF91CF911F910895809133038170089577
:1047500086E090E00C948434682F86E090E00C941E
:1047600098348091330384708962809333030C946E
:10477000AC238091330386958695869508950E9493
:104780005012811104C00E94FD120E94B1230E94A8
:10479000A82380933303282F26952695269530E06D
:1047A0002630310524F0877088628093330380912E
:1047B000330380FF04C086958695869501C080E00E
:1047C0000C943C2520913303822F869586958695FF
:1047D000482F50E04530510554F48F5F982F990FC2
:1047E000990F990F822F8770892B809333038091C3
:1047F00033038160809333030E94AC2380919C0239
:1048000080FF11C0809133038695869586951F920F
:104810008F938BED97E09F938F930E94F0050F90FD
:104820000F900F900F908091330386958695869513
:104830000C943C2580913303982F969596959695E8
:10484000A1F0915E990F990F990F8770892B809332
:104850003303887F91E009F490E08091330390FB6B
:1048600080F9809333030E94AC2380919C0280FFE7
:1048700011C0809133038695869586951F928F93FC
:1048800083EC97E09F938F930E94F0050F900F9019
:104890000F900F90809133038695869586950C94A2
:1048A0003C258091330380FD1FC0816080933303DA
:1048B000813019F489E080933303809133030E949F
:1048C000AC2380919C0280FF08C08BE997E09F9306
:1048D0008F930E94F0050F900F908091330386957F
:1048E000869586950C943C2508958091330380FF2E
:1048F00014C08E7F809333030E94AC2380919C026E
:1049000080FF08C088E897E09F938F930E94F0058E
:104910000F900F9080E00C943C250895CF93C091A8
:104920003303C17080919C0280FF0CC01F92CF9313
:104930008DEA97E09F938F930E94F0050F900F9060
:104940000F900F90CC2319F0CF910C947524CF9138
:104950000C94512490913303892F869586958695E2
:104960008F5F8F719770863038F4880F880F880FAB
:10497000892B8093330302C09093330380913303D8
:10498000887F91E009F490E08091330390FB80F9F7
:10499000809333030E94AC2380919C0280FF11C05E
:1049A000809133038695869586951F928F9384E731
:1049B00097E09F938F930E94F0050F900F900F90B8
:1049C0000F90809133038695869586950C943C25AF
:1049D000863008F085E0909133039770282F220FDE
:1049E000220F220F922B90933303987F21E009F43A
:1049F00020E09091330320FB90F9909333030C94C3
:104A00003C250E94E824809133030C94AC239C0144
:104A1000FB018281882349F12E3BFCE53F07C9F069
:104A200040F42C3BECE53E0769F02D3B3C4561F042
:104A30000895203C9CE5390791F070F0213C3C45FD
:104A400089F0089585E001C080E00E94012580E0A2
:104A500008950E941A24FBCF0E94E223F8CF0E94FF
:104A60008E24F5CF0E94AA24F2CF81E00895269AE1
:104A70002E9808952E9808958F929F92AF92BF928C
:104A8000CF92DF92EF92FF920F931F93CF93DF931A
:104A9000C82F863050F4811109C0809180008F7D2D
:104AA000809380000E943A2506C0C5E08091800076
:104AB000806280938000A0918600B09187002C2FA7
:104AC00030E00E94383425E030E040E050E00E94C1
:104AD00008340027122F232F342F012F122F232FBA
:104AE000332780918600909187006CE070E00E94EF
:104AF000E0336017710730F0C80169E070E00E9490
:104B0000E0335EC08091860090918700E09086003F
:104B1000F0908700E0918600F0918700C6E0D0E039
:104B2000BE010E94E033060F171F211D311D4801F1
:104B3000590185E0880C991CAA1CBB1C8A95D1F7E9
:104B4000C701BE010E94E0336F01E12CF12CA701E7
:104B50009601260F371F411D511DC501B4010E944A
:104B6000083469017A01E0918600F0918700CA015A
:104B7000B9010E94B6339B01AC01DF010E944E34A3
:104B80009B01AC01C701B6010E94B633DC01CB0129
:104B90002FE0B695A795979587952A95D1F700911F
:104BA00086001091870020E030E0081719072A07D7
:104BB0003B0728F46091860070918700CB01BC010F
:104BC00070938B0060938A00DF91CF911F910F91BA
:104BD000FF90EF90DF90CF90BF90AF909F908F901D
:104BE000089508950E94372582E28093800089E12C
:104BF000809381008FEF9FEF9093870080938600D2
:104C00000C94BF23539A2BB1277F3BB138604FB729
:104C1000F894FC01CB01880F991F680F791F6E0F64
:104C20007F1FE617F70789F0819198E03BB90000F4
:104C300000C087FF2BB9880F000000C000C000C073
:104C40002BB900C09A9591F7ECCF4FBF8FE594E058
:104C50000197F1F700C0000008950895FC01680F66
:104C6000791F8FEF91E3E617F70771F02191822703
:104C700028E030E087FF03C0880F892701C0880F34
:104C800021503109B9F7EFCF0895CF93DF93EC01AD
:104C9000FB018281882309F43CC1C430FDE5DF07B4
:104CA00060F4CB3F9CE5D90788F49E0122503C4537
:104CB0002431310508F02EC109C0C236EDE5DE070A
:104CC00029F0C63AFDE5DF0709F024C10E94681209
:104CD0009093F3028093F202C1318CE5D80709F476
:104CE000C6C008F042C0C930ECE5DE0709F49BC03D
:104CF00000F5C5308CE5D80709F485C078F4C330D9
:104D0000ECE5DE0709F478C008F07AC0C230DC4573
:104D100009F0F5C08091F2028160EFC0C7309CE5D8
:104D2000D90709F478C008F07AC08091F202806156
:104D3000E4C0CD30FCE5DF0709F487C058F4CB3080
:104D40009CE5D90709F479C008F07BC08091F20294
:104D500088606FC0CF30FCE5DF0709F480C008F041
:104D600082C08091F202877FC8C0CE3F9CE5D90700
:104D700009F471C000F5C531FCE5DF0709F485C011
:104D800068F4C3319CE5D90709F475C008F095C0F3
:104D90000E94040C8091F2028F77AFC0CC3FFCE5FB
:104DA000DF07A9F108F054C0CB3FDC4509F0A7C0EC
:104DB0008091F30240C0C230EDE5DE0709F489C0FE
:104DC00058F4C1158DE5D80709F45AC008F069C038
:104DD0008091F30282602FC0C236EDE5DE0709F450
:104DE0007CC0C63AFDE5DF0709F481C0C330DD456C
:104DF00009F085C080E06EC08091F20282607DC0C3
:104E00008091F20216C08091F202886076C0809193
:104E1000F30282604FC08091F20280626EC0809186
:104E2000F20280646AC00E94040C8091F2028068E1
:104E300064C0846062C081603DC08091F2028E7F58
:104E40005CC08091F2028D7F58C08091F20216C042
:104E50008091F30218C08091F3028D7F2BC0809166
:104E6000F2028F7E4AC08091F2028F7D46C080910F
:104E7000F2028F7B42C08091F202877F8B7F3DC020
:104E80008091F3028D7F8E7F15C08091F20282FBAC
:104E9000222720F991E0922790FB82F990FB83F979
:104EA0002CC08091F302982F909591708E7F892B62
:104EB00090FB81F98093F30222C00E94040C809140
:104EC000F20287FB222720F991E0922790FB87F9D5
:104ED00014C081E00E94091312C08091F20284FB89
:104EE000222720F991E0922790FB84F906C0809157
:104EF000F202982F909590FB80F98093F2028091B6
:104F0000F2029091F3020E9479120E94040C80E058
:104F100001C081E0DF91CF910895CF93DF93863177
:104F20009C4541F5EB010E945911982F8A812091EF
:104F3000020130910301882379F09A7A81E009F423
:104F400080E08093D102911102C069E201C065E363
:104F5000C9010E94192B0AC08091D102811102C09F
:104F600069E201C065E3C9010E941B2B0E949B11ED
:104F700080E001C081E0DF91CF9108950F931F93EE
:104F8000CF93DF93C42FD22FFC0182818823C9F0F5
:104F90004093D4020E94BF2B9093D3028093D202FD
:104FA00080E28C0F883008F057C0C77081E001C0E4
:104FB000880FCA95EAF7DF91CF911F910F910C945A
:104FC00070098091D402481330C08091D202909130
:104FD000D3020E94D72B883C910538F510E21D0FB3
:104FE000CD17B9F080E28C0F883040F4C77081E0B3
:104FF00001C0880FCA95EAF70E947709183028F592
:1050000081E09D2F977001C0880F9A95EAF70E9462
:105010007009802F0E9467091830F0F4D77081E082
:1050200001C0880FDA95EAF70AC080E28C0F883059
:1050300098F4C77081E001C0880FCA95EAF7DF9144
:10504000CF911F910F910C947709802FDF91CF9111
:105050001F910F910C946709DF91CF911F910F91D0
:1050600008950F939C01CB01243F4CE5340731F1A7
:1050700088F4293DFCE53F07D9F02A3D4CE534078B
:1050800079F1283D3C45A9F506E221EE41EE68EDB7
:105090007CE52BC0263FFCE53F07E1F0A8F0273F69
:1050A0003C4539F507E225EE46EE67EF7CE51DC08D
:1050B00007E225EE45EE69ED7CE517C006E221EE3C
:1050C00040EE64EF7CE511C007E225EE44EE65EFAB
:1050D0007CE50BC006E221EE42EE66EF7CE505C002
:1050E00008E221E045EE6AED7CE50E94BE2780E003
:1050F00008C0FC018281882319F01092D40201C0FB
:1051000081E00F9108958EE1489B02C08150E1F744
:10511000489BFECF0895589880E28A95F1F7589AF7
:105120000895FC012AE02A95F1F728E090E080E05C
:1051300031E040E14A95F1F7880F489B02C0816059
:10514000932700C0000040E14A95F1F7215089F70C
:1051500020E12A95F1F729B100C0000030E13A952D
:10516000F1F7217092272081920F90830895EF929A
:10517000FF920F931F93CF93DF931F92CDB7DEB7AC
:1051800019828C017C01E60EF11C0E151F0551F0F1
:105190000E948328CE0101960E949128F8018193F4
:1051A0008F01F3CF81E09981911180E00F90DF9121
:1051B000CF911F910F91FF90EF900895509A589AB8
:1051C00008955098589AE89AE9E6F0E080818C7F3B
:1051D00080830895615091E001C0990F6A95EAF7C4
:1051E00020E031E0992361F0492F482319F0589AC3
:1051F000232701C0589840E24A95F1F79695F2CFDF
:10520000222311F0589A01C0589880E28A95F1F74C
:1052100058980895FF920F931F93CF93DF93EC015B
:105220008C01060F111DC017D10741F0F9900E94A3
:105230008B2868E08F2D0E94EA28F5CFDF91CF916F
:105240001F910F91FF9008951F920F920FB60F922A
:1052500011240F931F932F933F934F935F936F935B
:105260007F938F939F93AF93BF93EF93FF93CF93CE
:10527000DF931F92CDB7DEB719820E948328CE013B
:1052800001960E949128082F069506950695902F65
:1052900096959570202F2570920F292F2370969543
:1052A0009695920F877089135FC0898181115CC0C8
:1052B000053008F059C080E18A95F1F7589A509A64
:1052C00082E08A95F1F700C0589888E0089F800135
:1052D0001124D801AB5FBE4F1696ED91FC91179744
:1052E0003097A9F06091B2017091B30114962D919D
:1052F0003C911597260F371F11968D919C9112970F
:10530000680F791F13964C9113978C910995F801AA
:10531000EB5FFE4F6381662351F08091B201909163
:10532000B30124813581820F931F0E940A290E94B4
:105330008B2880E18A95F1F758985098589A80E127
:105340008A95F1F7F801EB5FFE4F6081662351F01B
:105350008091B2019091B30121813281820F931F1C
:105360000E94B7280E9483280F90DF91CF91FF9170
:10537000EF91BF91AF919F918F917F916F915F91CD
:105380004F913F912F911F910F910F900FBE0F9052
:105390001F9018950F931F93CF93DF93853091053E
:1053A0000CF06DC0EC01F894509A589885E08A95FD
:1053B000F1F700009C2F969595702C2F2570920F79
:1053C000892F83709695969523E0CC0FDD1F2A9543
:1053D000E1F7980F8E01092B0E948B2884E08A95B3
:1053E000F1F700C068E0802F0E94EA2880E18A95EA
:1053F000F1F75098589A489902C000C0FCCF87E056
:1054000090E0489B08C0019721F4509A589A7894EC
:1054100036C000C0F6CFFE01EB5FFE4F638166230E
:1054200081F08091B2019091B30124813581820F86
:10543000931F0E94B728811104C0509A589A7894FB
:105440001FC00E94832880E28A95F1F75898509AED
:1054500080E18A95F1F7CB5FDE4F6881662351F0DA
:105460008091B2019091B30129813A81820F931FFB
:105470000E940A290E948B28789481E001C080E074
:10548000DF91CF911F910F91089590930B0280931C
:105490000A0208959093DB028093DA0208950E9435
:1054A0006018811103C08091D5020895E091DA025D
:1054B000F091DB02309721F00190F081E02D09940A
:1054C00080E00895EF92FF920F931F93CF93DF93A5
:1054D000E091DA02F091DB023097B1F18C010280A9
:1054E000F381E02D099580919C0282FF2DC080FF01
:1054F00004C08BEF98E00E945705E80118E085EFA3
:10550000E82E88E0F82E80919C0280FF0BC08881F5
:105510001F928F93FF92EF920E94F0050F900F90D1
:105520000F900F90115021961111EDCF80919C0298
:1055300080FF0AC083EF98E0DF91CF911F910F9118
:10554000FF90EF900C945705DF91CF911F910F9131
:10555000FF90EF9008952091D8023091D90228173A
:10556000390771F09093D9028093D802E091DA0262
:10557000F091DB02309721F00680F781E02D09944D
:1055800008952091D6023091D7022817390771F07B
:105590009093D7028093D602E091DA02F091DB0279
:1055A000309721F00084F185E02D09940895FC01E5
:1055B000329697E080E0915029F021912223D9F38F
:1055C0008F5FF9CF0895662349F0FC013296089663
:1055D0002191621729F0E817F907D1F780E00895C3
:1055E00081E008959C01FC0132969FEF80E041919B
:1055F000461789F09F3F19F4411101C0982F8F5F22
:105600008630A9F79F3F39F0F901E90FF11D97FDA9
:10561000FA956283089508959C012A5F3F4FFC012B
:105620004281461301C01282019682179307B9F78F
:1056300008950C94F22A0C940C2B029626E0FC019F
:1056400011922A95E9F7089508950C94242B83E08C
:105650008093DC020C94252B811102C081E001C0F3
:1056600082E08093DC020C94252B0C942C2B81E09F
:105670008093DC020C94252B0C94372B08950C940A
:105680003E2B0C943F2B0C943E2B0C943E2B0C94F5
:105690003E2BCF930E94452B0E94D3170E94432B91
:1056A000C0E08C2F0E944F16811104C0CF5FCA301A
:1056B000C1F701C081E0CF91089508951F920F9224
:1056C0000FB60F9211248F939F93AF93BF93809146
:1056D000DD02811113C08091340390913503A091B4
:1056E0003603B09137034196A11DB11D8093340359
:1056F00090933503A0933603B0933703BF91AF91D6
:105700009F918F910F900FBE0F901F9018958091D1
:105710003C03843031F10E9496071092DD0220E4B0
:1057200088E190E00FB6F894A895809360000FBED2
:105730002093600083B7817F846083BF83B78160DB
:1057400083BF7894889583B78E7F83BF0FB6F89414
:10575000A89580916000886180936000109260003D
:105760000FBE08950E94040C0C949D0782E084BD36
:1057700093E095BD9AEF97BD80936E0008952FB783
:10578000F8948091340390913503A0913603B09141
:1057900037032FBF08952FB7F894609134037091A9
:1057A000350380913603909137032FBF08959C01F4
:1057B0004FB7F8948091340390913503A09136034C
:1057C000B09137034FBF821B930B0895CF92DF92A6
:1057D000EF92FF922FB7F894C0903403D090350326
:1057E000E0903603F09037032FBFA7019601261BE8
:1057F000370B480B590BCA01B901FF90EF90DF90AE
:10580000CF90089578941F920F920FB60F921124A3
:105810008F939F93AF93BF938091340390913503FF
:10582000A0913603B09137030196A11DB11D80935D
:10583000340390933503A0933603B0933703BF919D
:10584000AF919F918F910F900FBE0F901F90189561
:1058500087E797E790930108809300089AE088E132
:105860000FB6F894A895809360000FBE90936000E7
:10587000FFCF8091EC0208950895CF93DF9321E04C
:105880002093E9002FEF3091E800215035FD06C04C
:1058900035ED3A95F1F700002111F5CF2091E800A0
:1058A00025FF14C0EC0140E050E068E070E00E9489
:1058B000072F8091E8008E778093E80088E0FE0152
:1058C000A4EEB2E001900D928A95E1F7DF91CF91BD
:1058D00008958093E0027093E2026093E102809168
:1058E0003C03843001F582E08093E9008FEF9091D2
:1058F000E800815095FD06C095ED9A95F1F70000FE
:105900008111F5CF8091E80085FF0DC040E050E0A7
:1059100063E070E080EE92E00E94072F8091E80043
:105920008E778093E8000895BC0184E00C94692C84
:10593000BC0183E00C94692C089581E299E00E94F7
:10594000570580913B03811109C00E9498300E9445
:10595000F5308091E20084608093E20008958DE14B
:1059600099E00E94570510923B03089589E199E060
:105970000E9457050C943C2B85E199E00E94570545
:105980006091380381E0611101C080E00C94272B05
:1059900081E199E00E94570590913C0381E09430A9
:1059A00009F080E0609138030C942C2B2091DF02E9
:1059B0002F5F822F62E30E94C633992319F0209350
:1059C000DF0208951092DF028091E302882371F1D3
:1059D00080913C03843041F58091E9008F702091E3
:1059E000EC00922F917020FD90E8892B93E090932A
:1059F000E9009091EB0090FF14C09091EE0097FFAA
:105A000010C09091E80095FF03C01092F100F9CF0B
:105A10009091E80090FF05C09091E8009E779093E8
:105A2000E8008F708093E9001092E302089542E04D
:105A300061EC81E00E94113042E261EC82E00E9460
:105A4000113042E261EC83E00E94113090913C03FE
:105A500081E0943009F080E0609138030C94352B9C
:105A600080913E03833009F461C030F4813071F0DD
:105A7000823009F49AC008958A3009F486C08B30C8
:105A800009F46CC0893009F0A8C020C080913D03A2
:105A9000813A09F0A2C08091E800877F8093E800F6
:105AA0008091410390914203892B21F468E084EEB8
:105AB00092E003C060E080E090E070E00E94522F2E
:105AC0008091E8008B778093E800089580913D03F2
:105AD000813209F082C08091410390914203029784
:105AE00008F07BC08091E800877F8093E800809178
:105AF000E80082FD05C080913C038111F8CF6DC0A4
:105B00002091F3008091F20090E0922B029731F403
:105B10008091F100813011F0863021F48091F10004
:105B20008093EC028091E8008B7753C080913D0315
:105B3000813A09F052C08091410390914203892B30
:105B400009F04BC08091E800877F8093E800809146
:105B5000E80080FFFCCF8091440136C080913D0376
:105B60008132D9F58091410390914203892BA9F5A7
:105B70008091E800877F8093E8000E944630809102
:105B80003F03809344010C94040C80913D038132C7
:105B900021F58091E800877F8093E8000E944630DD
:105BA000809140038093ED02089580913D03813AF6
:105BB000A1F48091E800877F8093E8008091E8005D
:105BC00080FFFCCF8091ED028093F1008091E8008E
:105BD0008E778093E8000C94463008959FB7F89430
:105BE0001092E3029FBF90913C03943009F057C09C
:105BF0009091E9009F703091EC00232F217030FDCF
:105C000020E8922B23E02093E9002091EB0020FF75
:105C100043C02091EE0027FF3FC02091DE022223E7
:105C200021F02091E80025FF37C01092DE0226E027
:105C30003091E80035FD15C030913C03343061F5FA
:105C40003091EB0035FD28C0215021F481E0809394
:105C5000DE0222C0EFE9FFE03197F1F700C000005B
:105C6000E7CF8093F1008091E80085FD0AC0809124
:105C7000E80080FFFCCF8091E8008E778093E800F9
:105C800006C08FB7F89421E02093E3028FBF9F7086
:105C90009093E90080E008959F709093E9008FEF62
:105CA000089584B7877F84BF0FB6F894A895809134
:105CB0006000886180936000109260000FBE90E0E9
:105CC00080E80FB6F89480936100909361000FBE56
:105CD0000C94372B0E9498300E94F530E2EEF0E0F1
:105CE00080818460808378940C94893388E391E088
:105CF0000C944A2A80913C038530C9F48DE099E0E8
:105D00000E94570580913C03853079F40E94872BCF
:105D100080913A038823B1F30E94492B882391F3A1
:105D20000E94F12E0E94040CEDCF0C94B22B08952A
:105D300008950C949B2E292F332723303105C9F069
:105D400060F42130310581F02230310509F041C085
:105D50008BE590E027E539E040C021323105E1F0E4
:105D60002232310531F135C082E190E022EB39E099
:105D700034C099278130910549F028F0029749F500
:105D8000E5E2F9E005C0E3E5F9E002C0E3E4F9E0AB
:105D9000849190E09F0121C063307105D0F4660FBB
:105DA000771FFB01EC5FFD4F2081318189E090E09E
:105DB00014C06330710568F4FB01EE0FFF1FE25061
:105DC000FE4F20813181FB01E550FE4F808190E044
:105DD00004C080E090E020E030E0FA0131832083CD
:105DE000089580E189BD82E189BD09B400FEFDCF3F
:105DF0008091D8008F7D8093D8008091E0008260F0
:105E00008093E0008091E00081FDFCCF0895CF9267
:105E1000DF92EF92FF920F931F93CF93DF93EC01EA
:105E20008B017A010E946530811133C0E114F104C5
:105E300039F0F70180819181081B190BC80FD91F18
:105E4000C12CD12C0115110519F18091E80085FDB7
:105E500016C08091E8008E778093E800E114F10489
:105E600049F0F70180819181C80ED91ED182C0828C
:105E700085E00FC00E946530882321F30AC0899114
:105E80008093F10001501109FFEFCF1ADF0ADACF3A
:105E900080E0DF91CF911F910F91FF90EF90DF9005
:105EA000CF9008952091430330914403261737077C
:105EB00048F06115710539F42091E8002E772093A0
:105EC000E80001C0B901FC0120E06115710579F11C
:105ED00080913C038823F1F18530F1F18091E80055
:105EE00083FD3CC08091E80082FD2EC08091E800D7
:105EF00080FFEBCF2091F3008091F20090E0922B95
:105F00006115710551F08830910538F42191209385
:105F1000F100615071090196F3CF21E0089709F073
:105F200020E08091E8008E778093E800CECF2111A9
:105F3000CFCF0AC080913C03882361F0853061F0A7
:105F40008091E80083FD0AC08091E80082FFF2CFD3
:105F500080E0089582E0089583E0089581E0089547
:105F600020914303309144032617370748F0611509
:105F7000710539F42091E8002E772093E80001C0E4
:105F8000B901FC0120E06115710591F180913C039C
:105F9000882309F440C0853009F43FC08091E800AF
:105FA00083FD3DC08091E80082FD2FC08091E80014
:105FB00080FFE9CF2091F3008091F20090E0922BD6
:105FC0006115710559F08830910540F424912093B2
:105FD000F1003196615071090196F2CF21E00897E6
:105FE00009F020E08091E8008E778093E800CBCF25
:105FF0002111CCCF0AC080913C03882361F0853009
:1060000061F08091E80083FD0AC08091E80082FF82
:10601000F2CF80E0089582E0089583E0089581E062
:106020000895982F973068F59093E900981739F004
:106030007091EC002091ED005091F00003C0242FEE
:10604000762F50E021FD02C09F5FECCF3091EB0036
:106050003E7F3093EB003091ED003D7F3093ED00BB
:106060003091EB0031603093EB007093EC002093A3
:10607000ED005093F0002091EE0027FDE5CF80E089
:1060800008958F708093E90081E0089580913D0329
:1060900087FF11C08091E80082FD05C080913C031C
:1060A0008111F8CF11C08091E8008B770BC08091EF
:1060B0003C03882349F08091E80080FFF8CF80916D
:1060C000E8008E778093E80008952091E4003091F5
:1060D000E50095E64091EC00842F817040FF23C0DD
:1060E0008091E80080FD1DC080913C03882399F0D9
:1060F000853099F08091EB0085FD11C04091E4005E
:106100005091E5002417350729F3915011F09A01B9
:10611000E1CF84E0089582E0089583E0089581E06E
:10612000089580E008954091E80042FFDDCF089592
:106130000E9406310E940E31E0EEF0E08081816025
:106140008083E8EDF0E080818F77808319BCA7ED34
:10615000B0E08C918E7F8C9380818F7E80831092B3
:106160003B0308950F931F93CF93DF930E94063153
:106170000E940E31C8EDD0E088818F7788838881B6
:106180008068888388818F7D888319BC10923C0346
:106190001092380310923A031092390300EE10E087
:1061A000F80180818B7F808388818160888342E0D1
:1061B00060E080E00E941130E1EEF0E080818E7FAF
:1061C0008083E2EEF0E0808181608083808188605E
:1061D0008083F80180818E7F8083888180618883BD
:1061E000DF91CF911F910F910895E8EDF0E080814C
:1061F0008F7E8083E7EDF0E080818160808384E0A2
:1062000082BF81E080933B030C94B230E8EDF0E074
:1062100080818E7F80831092E20008951092DA00D0
:106220001092E10008951F920F920FB60F92112461
:106230002F933F934F935F936F937F938F939F938E
:10624000AF93BF93EF93FF938091E10082FF0BC068
:106250008091E20082FF07C08091E1008B7F8093F4
:10626000E1000E94D62C8091DA0080FF1FC080914F
:10627000D80080FF1BC08091DA008E7F8093DA0007
:106280008091D90080FF0DC080E189BD82E189BD88
:1062900009B400FEFDCF81E080933C030E949D2C59
:1062A00005C019BC10923C030E94AF2C8091E10004
:1062B00080FF19C08091E20080FF15C08091E2004C
:1062C0008E7F8093E2008091E20080618093E20003
:1062D0008091D80080628093D80019BC85E08093BB
:1062E0003C030E94BC2C8091E10084FF30C080916F
:1062F000E20084FF2CC080E189BD82E189BD09B440
:1063000000FEFDCF8091D8008F7D8093D8008091D2
:10631000E1008F7E8093E1008091E2008F7E809388
:10632000E2008091E20081608093E2008091380376
:10633000882311F084E007C08091E30087FD02C04C
:1063400081E001C083E080933C030E94C82C8091CF
:10635000E10083FF29C08091E20083FF25C0809186
:10636000E100877F8093E10082E080933C031092FC
:1063700038038091E1008E7F8093E1008091E200FC
:106380008E7F8093E2008091E20080618093E20042
:1063900042E060E080E00E9411308091F00088606F
:1063A0008093F0000E94B62CFF91EF91BF91AF91C6
:1063B0009F918F917F916F915F914F913F912F911D
:1063C0000F900FBE0F901F9018951F920F920FB64F
:1063D0000F9211242F933F934F935F936F937F936B
:1063E0008F939F93AF93BF93CF93DF93EF93FF93DD
:1063F000C091E900CF708091EC00D82FD17080FD62
:10640000D0E81092E9008091F000877F8093F0003F
:1064100078940E9429321092E9008091F0008860FF
:106420008093F000CD2BCF70C093E900FF91EF91E6
:10643000DF91CF91BF91AF919F918F917F916F919C
:106440005F914F913F912F910F900FBE0F901F9032
:1064500018951F93CF93DF93CDB7DEB7AA970FB6EA
:10646000F894DEBF0FBECDBFEDE3F3E08091F10005
:10647000819323E0E534F207C9F70E94302D809123
:10648000E80083FF2EC180913D0390913E03492F88
:1064900050E04A30510508F024C1FA01EE59FF4F8F
:1064A0000C942A34803821F0823809F01AC108C0CF
:1064B0008091390390913A03992389F082600FC04B
:1064C000809141038F70873008F00BC18093E90001
:1064D0008091EB0085FB882780F91092E90090916C
:1064E000E800977F9093E8008093F1001092F1000C
:1064F000D1C0282F2D7F09F0F4C0882319F08230F5
:1065000061F0EFC080913F03813009F0EAC0933021
:1065100009F080E080933A032EC080913F038111FF
:106520002AC0809141038F702FEF280F263008F08A
:10653000D8C08093E9002091EB0020FF1CC093306D
:1065400021F48091EB00806214C09091EB00906187
:106550009093EB0021E030E0A90102C0440F551FE9
:106560008A95E2F74093EA001092EA008091EB00EE
:1065700088608093EB001092E9008091E800877FAB
:106580008093E8000E944630ACC08111AAC01091EF
:106590003F031F778091E3008078812B8093E30095
:1065A0008091E800877F8093E8000E9446308091C8
:1065B000E80080FFFCCF8091E30080688093E300D7
:1065C000111102C082E001C083E080933C0389C0C6
:1065D0008058823008F085C080913F03909140033D
:1065E0008C3D53E0950779F583E08A838AE28983BD
:1065F0004FB7F894DE01139620E03EE051E2E32F1E
:10660000F0E050935700E49120FF03C0E295EF7053
:106610003F5FEF708E2F90E0EA3010F0C79601C018
:10662000C0968D939D932F5F243149F74FBF809182
:10663000E800877F8093E8006AE270E0CE0101966F
:106640000E94522F16C06091410370914203AE0127
:106650004F5F5F4F0E94992EBC01892B09F441C006
:106660009091E800977F9093E80089819A810E9439
:10667000B02F8091E8008B778093E80032C080389B
:1066800081F58091E800877F8093E800809138034E
:106690008093F1008091E8008E7772CF811121C044
:1066A00080913F039091400399270297D4F4809101
:1066B000E800877F8093E80080913F038093380350
:1066C0000E94463080913803811106C08091E3001A
:1066D00087FD02C081E001C084E080933C030E94FA
:1066E000172D8091E80083FF0AC08091E800877F22
:1066F0008093E8008091EB0080628093EB00AA9683
:106700000FB6F894DEBF0FBECDBFDF91CF911F91C2
:106710000895CF9380913C038823A1F0C091E900B4
:10672000CF709091EC00892F817090FD80E8C82B8C
:106730001092E9008091E80083FD0E942932CF7019
:10674000C093E900CF9108950E94983010923C03C5
:106750000895E8EDF0E08081806180838AE18A9588
:10676000F1F700C08091D90081700895DB018F930B
:106770009F930E944E34BF91AF91A29F800D911DB7
:10678000A39F900DB29F900D11240895991B79E05D
:1067900004C0991F961708F0961B881F7A95C9F7B1
:1067A0008095089587FB082E062687FD819567FD55
:1067B00061950E94C6330EF4919507FC819508956A
:1067C000AA1BBB1B51E107C0AA1FBB1FA617B70717
:1067D00010F0A61BB70B881F991F5A95A9F7809533
:1067E0009095BC01CD01089597FB072E16F40094F7
:1067F00007D077FD09D00E94E03307FC05D03EF4B6
:10680000909581959F4F0895709561957F4F08955C
:10681000A1E21A2EAA1BBB1BFD010DC0AA1FBB1FA4
:10682000EE1FFF1FA217B307E407F50720F0A21B16
:10683000B30BE40BF50B661F771F881F991F1A9483
:1068400069F760957095809590959B01AC01BD01AD
:10685000CF010895EE0FFF1F0590F491E02D0994EC
:106860000E943834332312F48A1B9B0B0C94493456
:10687000A29FB001B39FC001A39F700D811D112481
:10688000911DB29F700D811D1124911D08950E94CC
:106890003834B7FF0895821B930B08950E94383453
:1068A000A59F900DB49F900DA49F800D911D112464
:1068B0000895B7FF0C944E340E944E34821B930B04
:1068C0000895FC014150504030F001900616D1F778
:1068D0003197CF010895882799270895FB01DC019E
:1068E00004C08D910190801921F441505040C8F7A7
:1068F000881B990B0895FB01DC0102C001900D92E9
:1069000041505040D8F70895F999FECF92BD81BD0E
:10691000F89A992780B50895A6E1B0E044E050E0E8
:106920000C94BE34A8E1B0E042E050E00C94BE34D8
:10693000262FF999FECF92BD81BDF89A019700B438
:10694000021639F01FBA20BD0FB6F894FA9AF99AD8
:106950000FBE08950396272F0E9499340E94983401
:10696000252F0E949934242F0C9499340196272FB7
:106970000E9499340C949834DC01CB01FC01F99904
:10698000FECF06C0F2BDE1BDF89A319600B40D927B
:0C69900041505040B8F70895F894FFCF34
:10699C00C80080020100000001000000000000009F
:1069AC0005010000000406000000000000010A00C0
:1069BC000000000000010102000C000C0C01191A6F
:1069CC001B1C1D1E1F202122392C3D2C9C2C982C6D
:1069DC00942C3C2C01E200E900EA00B500B600B7AB
:1069EC0000CD008301CC008A019201940121022385
:1069FC000224022502260227022A02B300B4006FE9
:106A0C00007000818283E200E900EA00B500B60064
:106A1C00B700CD008301CC008A01920194012102C0
:106A2C00230224022502260227022A02B300B40004
:106A3C006F007000818283F6F7313332F497C634DD
:106A4C003594A502736C6176655F6D6174726978BB
:106A5C000073796E635F74696D6572006261636B5C
:106A6C006C696768740000010202020206060609DE
:106A7C0009090909090F0F0F0F0F0F151515181913
:106A8C001919191919191919192324403222180A1C
:0A6A9C00E609C409690982099B0993
:00000001FF
